:020000040800F2
:1000000090AF0020DD010008D7420008A13D0008A4
:10001000D5420008650D0008B98500080000000001
:100020000000000000000000000000004501000882
:100030005F13000800000000890100086D7F0008C0
:10004000F7010008F7010008F7010008F7010008B0
:10005000F7010008F7010008F7010008F7010008A0
:10006000F7010008F7010008F7010008F701000890
:10007000F7010008F9120008051300081113000821
:100080001D130008F7010008F7010008F701000838
:10009000F7010008F7010008F7010008F701000860
:1000A000F7010008F97F0008F7010008F7010008D0
:1000B000F7010008F701000805800008F7010008B3
:1000C000F7010008F7010008F7010008F701000830
:1000D000F701000881840008E984000851850008C0
:1000E000F7010008F7010008F7010008F701000810
:1000F00011800008F7010008F7010008F701000867
:10010000F7010008F7010008F7010008F7010008EF
:10011000F7010008F7010008F7010008F7010008DF
:10012000F7010008F7010008F7010008291300088B
:10013000DFF80CD000F09AFB00480047D98C00088B
:1001400090AF0020224B19680868B0E8F00F80F3E8
:100150000988BFF36F8F4FF0000080F311884EF0D5
:100160000D0E70470000000006480068006880F32C
:10017000088862B661B6BFF34F8FBFF36F8F00DFA1
:1001800000BF00BF08ED00E0EFF30980BFF36F8F01
:100190000F4B1A6820E9F00F106008B54FF05000BF
:1001A00080F31188BFF34F8FBFF36F8F0AF09AF877
:1001B0004FF0000080F31188BDE808401968086816
:1001C000B0E8F00F80F30988BFF36F8F704700BF6E
:1001D00098090020EFF3058070470000064880472B
:1001E00006480047FEE7FEE7FEE7FEE7FEE7FEE71C
:1001F000FEE7FEE7FEE7FEE7F57F000831010008B5
:10020000202A04DB203A21FA02F00021704721FA6B
:1002100002F3D040C2F120029140084319467047D2
:10022000A0F16101192900D82038704740EA010384
:100230009B0703D009E008C9121F08C0042AFAD29C
:1002400003E011F8013B00F8013B521EF9D2704760
:10025000D2B201E000F8012B491EFBD27047002208
:10026000F6E710B513460A4604461946FFF7F0FFB5
:10027000204610BDF0B480EA0102D40F4200B2EB78
:10028000410F02D20246084611464A0042D0C30D31
:10029000DDB2C1F3C752AD1A202D35DAC1F3160114
:1002A00041F4000204B15242C5F1200602FA06F1FF
:1002B0002A411044B3EBD05F23D0C4B1012DA0EB91
:1002C000C35009DCF0BC4FF0004202EAC352DBB27B
:1002D00000F5000000F026BA400000F1807000EB4D
:1002E000C350A0F1807040EAD170490009E049088C
:1002F00041EAC071A0EBC35000F50000400800EBDC
:10030000C350F0BC00F005BA6142012202EB41018A
:10031000001BF6E7F0BC704781F00041AAE780F0CF
:100320000040A7E780EA010210B502F00043400058
:1003300022D04A001FD0010E01EB1261C0F356001B
:10034000C2F3560240F4000042F40002A0FB022077
:1003500000047F39140400D0401C50EA124001D43C
:100360004000491EC2B20C0604EBD010401C4008ED
:10037000802A02D003E0002010BD20F001000029F7
:1003800000DA0020184310BD2DE9FE4F804681EAB7
:100390000300C00F0C46009021F0004123F00045FF
:1003A000B8EB0200A94105D24046214690461C46C2
:1003B0000B46024623F00040104347D0270DC7F3F9
:1003C0000A00C3F30A510290401A019040286BDAE8
:1003D000C3F3130040F4801B0098924620B1002321
:1003E000D2EB030A63EB0B0B01985946C0F14002B4
:1003F000504600F06DF906460D4650465946019AA2
:1004000000F075F910EB08006141002487EA1152F1
:1004100084EAE7731A4340D0009A62B3019A012A32
:100420004FEA075215DC001B61EB02014FF000425E
:1004300002EA0752CDE90042001C41F58011324624
:100440002B4600F0ACF903B0BDE8F08F40462146E2
:10045000F9E7001B61EB0201001C41F58013001855
:100460005B412018A2F5001747EB030140EAD57065
:10047000B6196D4111E06D084FEA360645EAC075C0
:100480004FEA0752001B61EB0201001C41F580118D
:1004900049084FEA30000019514132462B4603B05B
:1004A000BDE8F04F00F06CB9009801224000002335
:1004B000D0EB020263EBE073009821464FEAE07450
:1004C000B8EB000061EB0401E9E783F000435BE770
:1004D00081F0004158E72DE9FE4F81EA030404F062
:1004E000004421F0004100944FF0000B23F0004342
:1004F00050EA01045ED052EA03045BD0C3F30A540D
:10050000C1F30A552C44A4F2F3340194A0FB025425
:10051000C1F3130141F48011C3F3130343F48013B7
:1005200001FB024400FB034E840A970A44EA81540B
:1005300047EA8357A4FB076802958D0A05FB0785E8
:100540004FEA932C04FB0C542705029D4FEA0658F2
:1005500047EA1637B5EB08056EEB070C870E920ECF
:1005600047EA811742EA8312A7FB0201B6EB0B01AF
:1005700064EB00042B0D43EA0C335E1844EB1C5073
:10058000DA465146E7FB0201C5F313044FEA0B3389
:1005900043EA14534FEA0432019C43EA0603A4F1F0
:1005A0000C040294009CCDE900B400F0F8F803B00C
:1005B000BDE8F08F00200146F9E7C10F80EAE07046
:1005C0000844CA079623002100F0ACB89623002205
:1005D000114600F0A7B800F0004220F00040C10D25
:1005E000C0F3160040F400007F2901DA00207047B4
:1005F000962903DCC1F19601C84001E09639884094
:10060000002AF4D04042704770B5C1F30A5201F09D
:1006100000450024C1F3130140F2FF3341F480117F
:100620009A4201DA002070BD40F233439A42A2F2AE
:10063000334203DC5242FFF7E3FD00E090402C43DD
:10064000F1D0404270BD00F0004230F000400AD0CE
:10065000C10D01F56071C0F3160042EA0151C208F4
:1006600040071143704700200146704701F00043E6
:1006700030B421F0004150EA010206D00A0DA2F583
:100680006072C1F31301002A02DC30BC0020704705
:10069000440F44EAC104C100E01830BC00EBC25072
:1006A00000F037B830B50B46014600202022012467
:1006B00009E021FA02F59D4205D303FA02F5491B30
:1006C00004FA02F52844151EA2F10102F1DC30BD46
:1006D000202A04DB203A00FA02F100207047914002
:1006E000C2F1200320FA03F3194390407047202AF7
:1006F00006DBCB17203A41FA02F043EAE07306E04A
:1007000041FA02F3D040C2F1200291400843194659
:1007100070470029A8BF7047401C490008BF20F05F
:100720000100704710B4B0FA80FC00FA0CF050EAF7
:10073000010404BF10BC704749B1CCF1200421FA78
:1007400004F411FA0CF118BF012121430843A3EB73
:100750000C01CB1D4FEA00614FEA102042BF002080
:1007600010BC704700EBC35010440029A4BF10BC5C
:100770007047401C490008BF20F0010010BC7047C2
:1007800010B5141E73F1000408DA401C41F1000199
:1007900092185B411A4301D120F0010010BD2DE9F0
:1007A000F04D92469B4611B1B1FA81F202E0B0FAE7
:1007B00080F220329046FFF78BFF04460F4640EA56
:1007C0000A0041EA0B0153465A46084313D011462A
:1007D00053EA010019D0C8F140025046FFF710FD5E
:1007E00005460E46504659464246FFF771FF0843FC
:1007F00005D0012004E020463946BDE8F08D0020F8
:10080000054346EAE0762C4337430A986305E40A39
:10081000A0EB08000022FD0A44EA47540A3002D542
:1008200000200146E9E7010510196941DDE90845A5
:1008300000196941BDE8F04DA2E7000030B5041E83
:1008400071F1000404DB4FF00044404264EB01010D
:10085000141E73F1000405DB1C464FF000435242A6
:1008600063EB0403994208BF904230BD064C074D2C
:1008700006E0E06840F0010394E807009847103470
:10088000AC42F6D3FFF758FC88B80008A8B80008B7
:1008900070B58D1810F8014B14F0030201D110F857
:1008A000012B231106D110F8013B03E010F8016B76
:1008B00001F8016B521EF9D1ABB110F8012B04F015
:1008C0000C048A1A0C2C03D0A2EB84129B1C08E0A7
:1008D00010F8014BA2EB0422F8E712F8014B01F8E3
:1008E000014B5B1EF9D5A942D4D3002070BD000096
:1008F000064A302908D001EBC10102EBC101A1F584
:100900008051A1F88602704750807047402800202F
:10091000F0B54FF6FF74A04201D0A14201D12046AC
:10092000F0BD44F250677D00B84200DB281A40F663
:10093000E444A04200DD2046DFF8ACC04FF4FA7674
:10094000BCF80240A0EB040EB64502DD04F5FA70D7
:1009500005E0A4EB000EB64501DDA4F5FA70ACF895
:100960000200B94200DB691A012A13DD1F4F37F874
:100970001340A1EB040CB44502DD04F5FA7105E067
:10098000A4EB010CB44501DDA4F5FA7127F81310AE
:10099000921E12E0154F203F37F81340A1EB040CD4
:1009A000B44502DD04F5FA7105E0A4EB010CB44591
:1009B00001DDA4F5FA7127F813106AB10844A842C2
:1009C00002DBA0F50C40A03846F678118842A7DD7E
:1009D000A0F50C40A038F0BD081A44F25061C8429E
:1009E000F2DA2844F0E70000140300202028002059
:1009F0002DE9F047264C8A4607463F2802DDA7F13D
:100A0000400001E0A7F13000814600EBC9008046BC
:100A100004EBC00634F8380006EBC0051D48E8605A
:100A200045F8080F6088A0F57F41FF391FD0B4F961
:100A30000410491C08D00AF04002B6F904104B46D5
:100A4000921CFFF765FF286007EBC70004EBC000AE
:100A5000A0F58050B0F98602401C08D00AF02002B0
:100A6000B6F9061060884B46FFF752FF686034F80D
:100A70003800401C80B224F83800082802D3002136
:100A800024F838104FF0FF30F080B080BDE8F087D8
:100A900040280020786FFFFF2DE9F043DFF8A480A5
:100AA000012208F50E64A4F58C654FF0000CDFF808
:100AB000989041E0C2EBC20000EB800005EB4000E3
:100AC0000121A0F83AC0A0F83EC0A0F836C0A0F8B6
:100AD00032C0A389012B1FD1238913B1012B1AD056
:100AE0001AE002EBC20308EBC30303EBC10349F2B4
:100AF0008807DE68FE4202DC068F761C0687DE6809
:100B0000B5F8423077429F4201DC9E4203DD038EFE
:100B10005B1C038600E000BF491C0229D9DB838FE0
:100B2000B0F840108B4202D30121C18703E08C450D
:100B300001D3A0F836C0521C99F800008242B9DDFA
:100B4000BDE8F0834028002014030020F0B58BB0EE
:100B500005461C4E1C4C28216846FFF780FBB4F864
:100B60001D001A4F40BAADF80000207D062804D1C0
:100B700001223946684600F08DFC0122394668465C
:100B800000F07AFCBDF80000000A2874BDF80000EF
:100B90006874BDF80000A0F57F41FF3901D0A6F8C8
:100BA0006C00287C617F884206D1687CA17F8842E6
:100BB00002D1207D062802D000200BB0F0BD01201C
:100BC000FBE70000203100206232002050F00708CF
:100BD0002B4A10B52B4953880BB1012010BD147D51
:100BE0000023062C12D0B1F87A20EAB147217F22E7
:100BF0008174C274FF24047543758175C2750476CF
:100C000043768176C2760477437737E01C4801212A
:100C100051808C38927F0270062242708370C170BE
:100C200003710821417129E0B1F90020120E82748C
:100C3000B1F90020120CC2740A88120A02750A78EF
:100C40004275B1F92820120E8275B1F92820120CD4
:100C5000C2750A8D120A027691F828204276B1F9FF
:100C60005020120E8276B1F95020120CC276B1F8E3
:100C70005020120A027791F850104177002010BDE1
:100C800062320020983B0020F0B58BB01F4C282129
:100C90006846FFF7E4FA002501221D49684600F086
:100CA000EBFBBDF800004FF6FF760127B04201D004
:100CB000608000E0678008221649684600F0DCFB8F
:100CC00069460EE031F81500B04204D004EB45024D
:100CD000A2F8440003E004EB4500A0F844706D1C4A
:100CE000EDB22088A842EDD800200B4908E004EBC3
:100CF00040020B88B2F84420401C1A440A80C0B25B
:100D000022888242F3D80BB0F0BD000020310020D1
:100D100024F0070860E00708820900200F4810B59A
:100D2000017D062901D0002010BD01210C4C41801D
:100D3000817F2170062161701221A170C17FE17055
:100D400090F8200020716171A0710821204603F005
:100D500029F8010AE1712072012010BD62320020E1
:100D60001C320020FEE70000F0B58BB005461C4C9D
:100D700028216846FFF773FA00206E4605E0211827
:100D8000497F26F81010401CC0B2217E8142F6D85F
:100D9000207D144F062804D1EA7A3946304600F007
:100DA00079FBEA7A3946684600F066FB00F09CF869
:100DB00000210CE0621836F81100527F904202D0F8
:100DC000227D062A09D06A18491C1074C9B2207EF7
:100DD0008842EFD801200BB0F0BD0020FBE70000F7
:100DE0006232002000F007082DE9F0470E46354C2E
:100DF0001546FFF728FC344A344BFFF769FB894658
:100E000007464FF03F4A012D43D0022D4CD04046BB
:100E1000FFF719FC3A464B46FFF75AFBFFF726FC53
:100E20002B49FFF77FFAFFF70EFC8A46074607F0CB
:100E3000E5FE89460546FFF7E7FB0446C62800DDC8
:100E4000C62436F81400FFF7C1FB804606EB4400C9
:100E50004088FFF7BBFB4146FFF75EFAFFF7F3FB65
:100E600004460E462A464B4638465146FFF72DFBB0
:100E700022463346FFF72FFB04460D464046FFF758
:100E8000E2FB22462B46FFF77FFABDE8F047FFF76B
:100E9000EDBBE06CFFF7D7FB3A464B46FFF718FB7C
:100EA000FFF7E4FBE06209E0606FFFF7CCFB3A4636
:100EB0004B46FFF70DFBFFF7D9FB60655045AFD9F7
:100EC0005046ADE7183900201D5A643BDF4FFD3F07
:100ED0000000C842704770477047704770477047BE
:100EE00070477047704770472DE9F04FA3B0C9486D
:100EF0000090C9480190C54CDFF81493DFF81CB38B
:100F0000C74DDFF820A3802102A8FFF7A8F900272A
:100F10000622C54902A800F0AFFABDF808004FF656
:100F2000FF78404514D1C822C049C14800F0B2FA48
:100F3000C822C049C04800F0ADFAC822BF49C04825
:100F400000F0A8FAC822BF49BF4800F0A3FA032066
:100F50002080BDF80A000126404506D013E004EBCE
:100F600047007F1C8686A681BFB22088B842F6D88B
:100F70000CE004EB4701BDF80A008886BDF80A00C2
:100F80007F1CA081BFB22088B842F2D8BDF80C0007
:100F9000404500D100206081BDF80E0040454FF073
:100FA000000006D011E004EB40012682401C8E8236
:100FB00080B221888142F6D80AE004EB4002268202
:100FC000BDF80E10401C918280B221888142F4D875
:100FD000BDF8100040454FF0000006D011E004EBD2
:100FE00040016682401C8E8480B221888142F6D8FE
:100FF0000AE004EB40026682BDF81010401C9184A8
:1010000080B221888142F4D887490122203102A888
:1010100000F032FABDF80800404501D1268100E019
:10102000208181490122283102A800F025FABDF86B
:101030000800404500D100207B49A08001223031CA
:1010400002A800F019FABDF80800404501D1E68079
:1010500000E0E08008227D4902A800F00DFA00209F
:1010600002AF37F810104A1E072A02D204EB4002E2
:10107000918604EB4001401C80B28E860828F0D394
:10108000724908222039384600F0F6F9002037F876
:1010900010104A1E072A02D204EB4002918204EB90
:1010A0004001401C80B28E820828F0D36749082294
:1010B000203102A800F0E0F9002037F810104A1E95
:1010C000072A02D204EB4002918404EB4001401C49
:1010D00080B28E840828F0D353490122383102A807
:1010E00000F0CAF9BDF808004746B84202D1A4F89A
:1010F0006E6001E0A4F86E004B490122403102A865
:1011000000F0BAF9BDF80800B84200D10220A4F8F6
:10111000640004224E4902A800F0AEF9BDF80810A0
:101120004C48B94207D10021017041708170C170F3
:10113000E964696717E00A0AC2708170BDF80A1095
:101140000A0A427001700168E96400BFBDF80C1022
:101150000A0AC2708170BDF80E100A0A427001704E
:101160000068686700BF01222F4902A8483100F0DB
:1011700083F9BDF80800B84202D1A4F8666001E026
:10118000A4F8660028490122503102A800F074F941
:10119000BDF80800B84202D1A4F86C6001E0A4F8E0
:1011A0006C0021490122603102A800F065F9BDF808
:1011B0000800B84210D10520A9F886000099A1F8CE
:1011C0002C010199A1F84E00ABF87C002884AAF804
:1011D0007C0023B0BDE8F08FA9F88600A9F8CC0008
:1011E0000099A1F860000198BDF80810A0F84E1011
:1011F00000BFBDF80810ABF87C10BDF808002884CB
:10120000BDF80810AAF87C10E3E7000020310020A8
:10121000C02C0020B63200201C440020983B002047
:10122000183900201C3C002000F0070800D00708F7
:101230004003002000D40708D004002000D807088D
:101240006006002000DC0708F007002020E0070807
:1012500000C00708100100202DE9F05F2148224C52
:101260004FF48041C088214A214D224F4FF400495C
:101270008E114FF4007A4FF4006B08B101282FD182
:101280009046104601F050FCA4F8520049464046F2
:1012900001F04AFCA4F8A4004021284601F044FCD7
:1012A000A4F8F6008021284601F03EFCA4F848018D
:1012B0003146284601F038FCA4F89A0151462846E8
:1012C00001F032FCA4F8EC013146384601F02CFC68
:1012D000A4F83E025946384601F026FCA4F89002D4
:1012E000BDE8F09F203100201C440020000C01408C
:1012F0000010014000080140014801F0BDB80000A5
:1013000074270020014801F0B7B80000EC26002047
:10131000014801F0B1B80000940F0020014801F02D
:10132000ABB8000030270020014801F0A5B800004C
:10133000500F002030B590F840500124AC40C56BF0
:101340006C60046863604368102B036803D0996085
:101350000068C26030BD9A600068C16030BD7047EF
:1013600072B6FEE706490020C8610648016941F0EF
:1013700004010161016941F0400101617047000011
:10138000D80F002000200240064A0021D161064902
:101390000A6942F002020A614861086940F04000AF
:1013A00008617047D80F002000200240044B002243
:1013B000DA61044A136943F0010313610180704745
:1013C000D80F00200020024014490020CA68D3062C
:1013D000134A04D5D06940F00200D0611020CB68D8
:1013E0005B0705D5D36943F00103D36140F00400E6
:1013F000CB69DB0707D0D36943F00403D361CA6923
:1014000022F00102CA61A0F58072013A01D0C860E1
:101410007047C86920F00100C86170470020024091
:10142000D80F002070B5044601F090FB0546114E20
:1014300009E0601C07D024B101F088FB401BA042EA
:1014400001D9032070BDF068C007F2D1F0688006B2
:1014500001D52020F060F068C00605D4F069C0070F
:1014600002D1F068400703D5FFF7AEFF012070BD41
:10147000002070BD0020024010B507E011F8014BBC
:1014800011F8013B44EA032320F8023B521E92B2BA
:10149000F4D210BD2DE9F04786B00024C1F30A074D
:1014A00090468146CD1B0094019400BF0120CDE9F8
:1014B00003504FF4806A524629461448FFF7DCFF78
:1014C000124E06E039F8140004EB5701641C26F8AC
:1014D00011004445F6D301F01BFA00BF694601A88C
:1014E00001F076F900BF0024574636F8142005EBCA
:1014F00044010023012001F0C9F9641CA4B2BC42DC
:10150000F3D301F0B9F906B0BDE8F0870010002070
:101510002DE9F04F95B004460026DFF824943546B7
:1015200028216846FEF79BFE28210AA8FEF797FEB1
:101530006F460AAA09EB4600904630F8211F49BAC7
:1015400027F81610008840BA22F81600761CF6B26A
:10155000142EEFD399F81400062816D1F94E4FF641
:10156000FF71DFF8E4A3307C4FF0000901EA0020AE
:10157000717C4FF0010B0143B07C012906D0022998
:1015800079D0032978D0042977D0BEE3012812D07E
:1015900002283AD0032853D0042876D005286ED0EC
:1015A00006286DD007286CD008286BD009286AD08F
:1015B0000A2869D0A9E31422E4493846FFF76AFFF4
:1015C0001422E2496846FFF757FF0020414637F8EA
:1015D000103031F810209A4201D16D1CEDB2401C40
:1015E00080B21428F3D305E2022020751CE184F8B0
:1015F00014B019E1307C2074707C6074B07CA074ED
:10160000F07CE07484F814907FE3D04914222831F0
:101610003846FFF73FFFCD49142228316846FFF7CF
:101620002BFF0020414637F8103031F810209A4245
:1016300001D16D1CEDB2401C80B21428F3D39FE39E
:10164000C249142250313846FFF724FFBF49142203
:1016500050316846FFF710FF0020414637F8103040
:1016600031F810209A4201D16D1CEDB2401C80B2BD
:101670001428F3D3BEE1DBE00EE232E305E01FE025
:1016800039E053E06DE085E09FE0B0491422783105
:101690003846FFF7FFFEAD49142278316846FFF760
:1016A000EBFE0020414637F8103031F810209A4206
:1016B00001D16D1CEDB2401C80B21428F3D399E126
:1016C000A2491422A0313846FFF7E4FE9F491422B4
:1016D000A0316846FFF7D0FE0020414637F81030B1
:1016E00031F810209A4201D16D1CEDB2401C80B23D
:1016F0001428F3D37EE195491422C8313846FFF708
:10170000C9FE92491422C8316846FFF7B5FE002091
:10171000414637F8103031F810209A4201D16D1C43
:10172000EDB2401C80B21428F3D3FFE387491422A2
:10173000F0313846FFF7AEFE84491422F031684696
:10174000FFF79AFE0020414637F8103031F810209C
:101750009A4201D16D1CEDB2401C80B21428F3D323
:10176000E4E314227A493846FFF794FE14227849BC
:101770006846FFF781FE0020414637F8103031F807
:1017800010209A4201D16D1CEDB2401C80B2142889
:10179000F3D3CBE36E49142228313846FFF77AFEA3
:1017A0006B49142228316846FFF766FE0020414647
:1017B00037F8103031F810209A4201D16D1CEDB28B
:1017C000401C80B21428F3D3B0E361491422503195
:1017D0003846FFF75FFE5E49142250316846FFF736
:1017E0004BFE0020414637F8103031F810209A4265
:1017F00001D16D1CEDB2401C80B21428F3D3C4E3B8
:10180000BAF80000401C80B2AAF80000327C2274B2
:10181000727C6274B27CA274F27CE2740A287CD07E
:1018200084F814B0AAF80090012015B0BDE8F08F3C
:10183000012812D0022829D0032842D004285BD0E6
:1018400005286BD006286AD0072869D0082868D0F8
:10185000092867D00A2866D057E214223D49384645
:10186000FFF718FE14223B496846FFF705FE0020EB
:10187000414637F8103031F810209A4201D16D1CE2
:10188000EDB2401C80B21428F3D34FE33149142247
:1018900028313846FFF7FEFD2E49142228316846CC
:1018A000FFF7EAFD0020414637F8103031F81020EC
:1018B0009A4201D16D1CEDB2401C80B21428F3D3C2
:1018C0005EE22449142250313846FFF7E3FD2149F6
:1018D000142250316846FFF7CFFD0020414637F80B
:1018E000103031F810209A4201D16D1CEDB2401C2D
:1018F00080B21428F3D319E31649142278313846FC
:10190000FFF7C8FD1349142278316846FFF7B4FD8C
:101910000020414631F8102006E03BE31CE034E0B3
:101920004EE068E082E09CE037F810309A4201D146
:101930006D1CEDB2401C80B21428EBD3F6E200001F
:1019400062320020002200202403002000D007087B
:1019500018D1070800D407081422F9493846FFF7C0
:1019600099FD1422F6496846FFF786FD002041469E
:1019700037F8103031F810209A4201D16D1CEDB2C9
:10198000401C80B21428F3D3D0E2ED491422283150
:101990003846FFF77FFDEA49142228316846FFF7F1
:1019A0006BFD0020414637F8103031F810209A4284
:1019B00001D16D1CEDB2401C80B21428F3D3B5E206
:1019C000DF49142250313846FFF764FDDC49142208
:1019D00050316846FFF750FD0020414637F810307F
:1019E00031F810209A4201D16D1CEDB2401C80B23A
:1019F0001428F3D39AE2D249142278313846FFF7FB
:101A000049FDCF49142278316846FFF735FD0020A3
:101A1000414637F8103031F810209A4201D16D1C40
:101A2000EDB2401C80B21428F3D37FE2C4491422E3
:101A3000A0313846FFF72EFDC1491422A031684677
:101A4000FFF71AFD0020414637F8103031F810201A
:101A50009A4201D16D1CEDB2401C80B21428F3D320
:101A600064E2B7491422C8313846FFF713FDB44980
:101A70001422C8316846FFF7FFFC0020414637F8C2
:101A8000103031F810209A4201D16D1CEDB2401C8B
:101A900080B21428F3D378E2012812D0022829D08A
:101AA000032842D004285BD005287AD0062873D0BA
:101AB000072872D0082871D0092870D00A286FD062
:101AC00023E114229F493846FFF7E4FC14229D4984
:101AD0006846FFF7D1FC0020414637F8103031F856
:101AE00010209A4201D16D1CEDB2401C80B2142826
:101AF000F3D31BE29349142228313846FFF7CAFC7E
:101B00009049142228316846FFF7B6FC0020414670
:101B100037F8103031F810209A4201D16D1CEDB227
:101B2000401C80B21428F3D32AE186491422503194
:101B30003846FFF7AFFC8349142250316846FFF75F
:101B40009BFC0020414637F8103031F810209A42B3
:101B500001D16D1CEDB2401C80B21428F3D3E5E135
:101B60007849142278313846FFF794FC75491422DD
:101B700078316846FFF780FC0020414637F8103086
:101B800031F810209A4201D16D1CEDB2401C80B298
:101B90001428F3D3CAE104E01EE038E052E06AE022
:101BA00084E068491422A0313846FFF773FC654988
:101BB0001422A0316846FFF75FFC0020414637F849
:101BC000103031F810209A4201D16D1CEDB2401C4A
:101BD00080B21428F3D3A9E15A491422C8313846F7
:101BE000FFF758FC57491422C8316846FFF744FCF8
:101BF0000020414637F8103031F810209A4201D1C8
:101C00006D1CEDB2401C80B21428F3D38EE14D4917
:101C10001422F0313846FFF73DFC4A491422F031D6
:101C20006846FFF729FC0020414637F8103031F8AC
:101C300010209A4201D16D1CEDB2401C80B21428D4
:101C4000F3D373E1142240493846FFF723FC1422F2
:101C50003D496846FFF710FC0020414637F8103038
:101C600031F810209A4201D16D1CEDB2401C80B2B7
:101C70001428F3D35AE13449142228313846FFF7A7
:101C800009FC3149142228316846FFF7F5FB002092
:101C9000414637F8103031F810209A4201D16D1CBE
:101CA000EDB2401C80B21428F3D33FE12649142240
:101CB00050313846FFF7EEFB234914225031684675
:101CC000FFF7DAFB0020414637F8103031F81020DA
:101CD0009A4201D16D1CEDB2401C80B21428F3D39E
:101CE00053E1012813D0022832D003285DD0042804
:101CF0007DD0052875D0062874D0072873D0082811
:101D000072D0092871D00A2870D000208DE51422E5
:101D10000E493846FFF7BEFB14220C496846FFF710
:101D2000ABFB0020414637F8103031F810209A42C2
:101D300001D16D1CEDB2401C80B21428F3D3F5E044
:101D4000A0D4070800D8070818D9070800DC07083E
:101D5000142292493846FFF79DFB14228F496846AA
:101D6000FFF78AFB0020414637F8103031F8102089
:101D70009A4201D16D1CEDB2401C80B21428F3D3FD
:101D8000142D7FF437ACBAF80000401C80B2AAF8DA
:101D90000000317C2174717C6174B17CA174F17C90
:101DA000E17428287FF423AC1EE47C4914222831F6
:101DB0003846FFF76FFB7949142228316846FFF750
:101DC0005BFB0020414637F8103031F810209A4272
:101DD00001D16D1CEDB2401C80B21428F3D3A5E0F4
:101DE00005E01FE039E053E06DE087E0B3E06B49C8
:101DF000142250313846FFF74DFB68491422503108
:101E00006846FFF739FB0020414637F8103031F8BB
:101E100010209A4201D16D1CEDB2401C80B21428F2
:101E2000F3D383E05D49142278313846FFF732FB63
:101E30005A49142278316846FFF71EFB00204146BC
:101E400037F8103031F810209A4201D16D1CEDB2F4
:101E5000401C80B21428F3D368E050491422A0310A
:101E60003846FFF717FB4D491422A0316846FFF7AB
:101E700003FB0020414637F8103031F810209A4219
:101E800001D16D1CEDB2401C80B21428F3D34DE09B
:101E900042491422C8313846FFF7FCFA3F49142260
:101EA000C8316846FFF7E8FA0020414637F810309D
:101EB00031F810209A4201D16D1CEDB2401C80B265
:101EC0001428F3D332E035491422F0313846FFF7B5
:101ED000E1FA32491422F0316846FFF7CDFA0020CA
:101EE000414637F8103031F810209A4201D16D1C6C
:101EF000EDB2401C80B21428F3D317E01422284915
:101F00003846FFF7C7FA142225496846FFF7B4FAA6
:101F10000020414637F8103031F810209A4201D1A4
:101F20006D1CEDB2401C80B21428F3D3142D7FF445
:101F300061ABBAF80000401C80B2AAF80000317C06
:101F40002174717C6174B17CA174F17CE1740A2804
:101F50007FF44DAB28E71249142228313846FFF7A9
:101F600099FA0F49142228316846FFF785FA0020B4
:101F7000414637F8103031F810209A4201D16D1CDB
:101F8000EDB2401C80B21428F3D3142D3FF438ACCA
:101F9000FFF730BB0220207544E4000028DC07086E
:101FA00040DD070870B51C4D1A4C6878032801D035
:101FB00006282DD1A878022803D10521164801F062
:101FC000F1FE6878032823D12878012100EB8002F4
:101FD00002EB801004EB4000A0F5A040A0F8881BA5
:101FE0002878E97800EB800202EB801004EB4000D7
:101FF000A0F5A040A0F8001B2878297900EB80020A
:1020000002EB801004EB4000A0F5A040A0F8281BD4
:1020100070BD00003C49002000230020054900EB72
:10202000C00202EB401031F8100008B100207047E8
:10203000012070471C4400202DE9F0411E4D1D4C2D
:102040001E4F6879A979012641EA0028687803289B
:1020500001D0062808D1A878022805D10521164804
:1020600001F0A0FE404500D03E80287800EB001132
:10207000C1EBC01004EB4000A0F5E040A0F8B66151
:102080002878E97800EB0012C2EBC01004EB4000A6
:10209000A0F5E040A0F814112878297900EB00128F
:1020A000C2EBC01004EB4000A0F5E040A0F83C11EA
:1020B000BDE8F081DC5100200023002084090020CD
:1020C00030B538493648384C0978012201EBC10354
:1020D00003EB411100EB4101A1F580510025A1F86E
:1020E00010262178212935D0222933D0232901D067
:1020F00024292ED16378032B2BD101EBC10303EBF1
:10210000411100EB4101A1F58051A1F80A56217857
:1021100001EBC10303EB411100EB4101A1F580513B
:10212000A1F81026217801EBC10303EB411100EB6C
:102130004101A1F58051A1F83E25217801EBC103B1
:1021400003EB411100EB4100A0F58050A0F85E25A3
:1021500000BF30BD6378032BFBD101EBC10303EB60
:10216000411100EB4101A1F58051A1F80A562178F7
:1021700001EBC10303EB411100EB4101A1F58051DB
:10218000A1F810262178E27801EBC10303EB41119D
:1021900000EB4100A0F58050A0F8C025D8E7000072
:1021A0001C440020002000200023002010B5040063
:1021B00002D0607910B106E0012010BD002020712E
:1021C000204600F005F801206071002010BD0000DD
:1021D00008B500680649884208D10648416941F0BF
:1021E00040014161406900F04000009008BD0000DE
:1021F000003002400010024070B54379012B20D01E
:10220000012444710223037103681E6802F0100266
:1022100040F6FE759540AE43D1E900510D4395401F
:1022200035431D6003681D68C02191408D431D60CA
:10223000026813688B4313600471002141710846E2
:1022400070BD022070BD70B5040003D02079002558
:1022500010B105E0012070BD6571204600F008F85E
:1022600002202071256101202071002070BD000036
:10227000F0B585B0002406460094019402940394BE
:1022800000681A4988422ED11949C86940F00050A7
:10229000C861C86900F000500490886940F00400EB
:1022A00088618869202700F0040004900320CDE9AC
:1022B000007069460F4800F03FFB104D0E48286043
:1022C0001020C5E901048020E860400028618000FA
:1022D000EC61C5E90507284600F0F2F908B1FFF7FF
:1022E0003FF8F5606E6205B0F0BD0000007400407C
:1022F000001002400008014044040240500F00203A
:1023000010B590F821100022022905D00421816324
:1023100080F82020012010BD01680B6823F00E0317
:102320000B6001680B6823F001030B6090F84030EC
:10233000012404FA03F1C36B596080F8214080F84E
:102340002020104610BD00002DE9F05F90F821100C
:102350000024022903D004218163012485E001685F
:102360000A6822F00E020A6001680A6822F001027F
:102370000A603F4E3E4FB215DFF8F4C0DFF8F09030
:10238000DFF8ECA0DFF8E8B0DFF8E4E00168783FC0
:1023900013011502ACF1640CA9F15009AAF13C0A31
:1023A000ABF1280BAEF1140E4FF48018B14227D9CF
:1023B000B9420ED0614512D049451DD0514518D0C3
:1023C000594518D0714501D1424615E0294EB14218
:1023D00001D1012210E0274E1436B14201D1102262
:1023E0000AE0244E2836B14206D0224A3C329142BD
:1023F00001D11A4600E02A461E49091F0A602BE057
:10240000B94213D0614517D0494522D051451DD05E
:1024100059451DD0714501D142461AE0B14202D161
:102420004FF0807215E0134EB14201D1012210E04D
:10243000104E1436B14201D110220AE00D4E28365A
:10244000B14206D00B4A3C32914201D11A4600E01B
:102450002A46074980394A60012180F8211000216D
:1024600080F82010416B01B188472046BDE8F09FFD
:1024700080000240080402402DE9F05FC16B0B6848
:1024800001680A68046C4FF0040808FA04F8844DE7
:10249000844E854FDFF814C2DFF81492DFF814A2DF
:1024A000DFF814B2DFF814E218EA030F65D05FEA30
:1024B000427862D50A68920603D40A6822F00402C0
:1024C0000A60DFF8F0814FF48062016808F11408B7
:1024D00013011402414524D9A9420DD0B1420FD0B5
:1024E000B9421AD0614515D0494515D0514501D1A1
:1024F000120312E0594501D104220EE0714501D1C9
:1025000040220AE06D4D1435A94206D06B4A2832AC
:10251000914201D11A4600E022466749091F0A602C
:1025200029E0A94213D0B14215D0B94220D061456B
:102530001BD049451BD0514502D14FF4800217E012
:10254000414502D14FF0806212E0594501D1042289
:102550000EE0714501D140220AE0584D1435A942E0
:1025600006D0564A2832914201D11A4600E022464E
:102570004B4908394A60C16A71E04FF0020808FA15
:1025800004F818EA030F70D05FEA82786DD50A6804
:10259000920606D40A6822F00A020A60012180F835
:1025A0002110DFF810814FF40072016808F114085F
:1025B00013011402414524D9A9420DD0B1420FD0D4
:1025C000B9421AD0614515D0494515D0514501D1C0
:1025D000120312E0594501D102220EE0714501D1EA
:1025E00020220AE0354D1435A94206D0334A28325C
:1025F000914201D11A4600E022462F49091F0A6084
:1026000029E0A94213D0B14215D0B94220D061458A
:102610001BD049451BD0514502D14FF4001217E0A1
:10262000414502D14FF0007212E0594501D102221A
:102630000EE0714501D120220AE0204D1435A94257
:1026400006D01E4A2832914201D11A4600E02246A5
:10265000134908394A60002180F82010816A002956
:102660001CD0BDE8F05F0847FFE70825A5401D42E4
:1026700014D0120712D50A6822F00E020A6090F8F0
:102680004020C36B012101FA02F25A60816380F895
:102690002110002180F82010016BE0E7BDE8F09FD9
:1026A000080002401C00024030000240440002408A
:1026B000580002406C000240080402401C04024022
:1026C00030B560B11A4B01681422994209D2194BF6
:1026D0000B44B3FBF2F292000264174A0AE00120B5
:1026E00030BD134B5B420B44B3FBF2F29200026429
:1026F0000F4A083AC263022280F821200A6843F692
:10270000F0739A43F0E901342343D0E902452C43A6
:1027100023430469234344692343846923431343C4
:102720000B6000214163012242770177084630BDEA
:1027300008040240F8FFFDBF0000024070B50446E7
:1027400090F82000002501280CD0012084F82000FA
:1027500094F821600020012E06D084F82000022584
:10276000284670BD022070BD022684F82160A06357
:102770002068066826F0010606602046FEF7DAFDAE
:10278000E06A00282068016802D041F00E0106E0EE
:1027900021F0040101602068016841F00A01016034
:1027A0002068016841F001010160D9E770B5044675
:1027B00000F0CCF90546601C02D0044800780444BF
:1027C00000F0C4F9401BA042FAD370BD8C09002070
:1027D0002DE9F047054626480F460126017E0129CE
:1027E0000FD00121814601762868DFF888804CF2FD
:1027F0005034022808D0A2462046FEF713FEA8B1A6
:1028000031E00220BDE8F0872046FEF70BFE08BB52
:102810000120FEF7A7FD2046FEF704FED8F81010B1
:10282000064621F00401C8F810101CE04FF0FF30FC
:102830003860AC6811E02046FEF7A6FD5046FEF772
:10284000F1FDD8F81010060021F00201C8F81010B0
:1028500001D03C6007E004F50064D5E9020100EB1B
:10286000C120A042E7D8002189F818103046C9E7F6
:10287000D80F0020002002400348016941F0800188
:102880000161002070470000002002402DE9F05F48
:1028900005461D4888460024017E16461F4601292C
:1028A00009D00121814601764CF2503A5046FEF79C
:1028B000B9FD18B123E00220BDE8F09F012D02D040
:1028C000022D00D00425D346DFF840A015E02201F8
:1028D00030463946FDF794FC81B208EB4400FEF720
:1028E00065FD5846FEF79EFDDAF8102022F0010241
:1028F000CAF8102018B9641CE4B2AC42E7D3002235
:1029000089F81820D8E70000D80F002000200240E6
:10291000064900200A69120607D5054A4A60054A99
:102920004A600969090600D501207047002002406D
:1029300023016745AB89EFCD2DE9F84FDFF8C09152
:10294000002409F1040A0AF1040B23464FF00F0892
:102950000BF1040ECCE00127A7403A40BA4272D1F5
:10296000DFF8A0C14D68A5EB0C0665452BD00DDC4A
:10297000032D34D005DC35B3012D19D0022D2FD114
:102980001BE0112D16D0122D2AD119E0B6F5881FA3
:1029900019D006DCB6F5803F15D0B6F5801F1FD1E3
:1029A00011E0B6F5001F0ED0B6F5041F18D10AE0ED
:1029B000CB6815E0CB681B1D12E0CB6808330FE035
:1029C000CB680C330CE08B682BB1012B4FF0080364
:1029D00003D0476104E0042302E0076100E0002324
:1029E000FF2A01D8064601E000F104064FEA8405FB
:1029F00001D9A5F12005376808FA05FC27EA0C077C
:102A000003FA05F547EA050737604D68ED006ED516
:102A10003D4DAE6946F00106AE61AD6924F0030696
:102A200005F001050095394D7719BE68A5072D0FF2
:102A300008FA05FC26EA0C06DFF8D4C0604503D18D
:102A40004FF0000C25E052E0DFF8C8C0604502D12D
:102A50004FF0010C1DE0DFF8C0C0604502D14FF01F
:102A6000020C16E0DFF8B4C0604502D14FF0030C51
:102A70000FE0DFF8ACC0604502D14FF0040C08E075
:102A8000DFF8A0C0604502D14FF0050C01E04FF027
:102A9000060C0CFA05FC4CEA060CC7F808C04D6899
:102AA000D9F80060ED034D4601D5164300E096438A
:102AB0002E604D68DAF80060AD03554601D5164327
:102AC00000E096432E604D68DBF80060ED025D4645
:102AD00001D5164300E096432E604D68DEF8006095
:102AE000AD02754601D5164300E096432E60641C86
:102AF0000A6832FA04F57FF42EAFBDE8F88F0000C3
:102B000000040140000011100010024000000140CC
:102B100000080140000C0140001001400014014079
:102B200000180140001C01408068084000D00120CE
:102B30007047C26821EA02030A4043EA0241016188
:102B400070470AB1016170470904FBE701488068DA
:102B5000704700008C090020024881680278114407
:102B6000816070478C090020074810B5016841F06A
:102B700010010160032000F095F8002000F006F835
:102B800000F03EF8002010BD0020024000B50146D4
:102B900087B000222C2000F065F82C2000F054F8BB
:102BA0001348816941F400518161806905A900F4ED
:102BB00000500690684600F023F900F051F90D49E5
:102BC0000D4AB0FBF1F10D48491E0260416040F230
:102BD000E7320021C0E90321816000F053FB10B10E
:102BE000012007B000BD054800F09AFBF9E700009E
:102BF0000010024040420F0000340140B82700207E
:102C00000F4808B5816941F001018161816901F0D6
:102C100001010091C16941F08051C161C069002288
:102C200000F0805000900F21901E00F01BF8054925
:102C3000486820F0E06040F00070486008BD000087
:102C40000010024000000140002809DB00F01F02D4
:102C5000012191404009800000F1E020C0F80011FE
:102C600070470000F0B40E4B1B68C3F30223C3F19E
:102C70000704042C00D904241D1D072D01D20023B4
:102C800000E0DB1E012606FA04F56D1E0D409D4096
:102C90009E40761E164045EA0601F0BC05F0E0BDF8
:102CA0000CED00E0064A00F0070110684FF6FF0344
:102CB000184040EA012003490843106070470000B3
:102CC0000CED00E00000FA052DE9F0470D46040088
:102CD00067D0DFF81881D8F8000000F00700A8429C
:102CE0000CD2D8F8001021F007012943C8F80010D1
:102CF000D8F8000000F00700A84252D120683C4EEE
:102D0000810712D5400703D5706840F4E060706019
:102D10002078000703D5706840F4605070607068D8
:102D2000A16820F0F000084370602078C00727D029
:102D30006068012810D03168022810D08907002966
:102D40002FDA716821F0030101437160FFF7FEFE85
:102D5000074641F288390CE031688903EFE78901C1
:102D6000EDE7FFF7F3FEC11B494502D90320BDE89B
:102D7000F0877068616800F00C00B0EB810FF0D153
:102D8000D8F80010404601F00701A9420BD90168AC
:102D900021F0070129430160006800F00700A84204
:102DA00001D00120E3E72078400705D57068E1688D
:102DB00020F4E060084370602078000706D5706852
:102DC000216920F4605040EAC100706000F058F8BA
:102DD0007168084AC1F30311515CC8400649086094
:102DE00006480068FFF7D2FE0020C0E7002002403E
:102DF0000010024050B5000888090020900900200A
:102E00000F2202600C4A536803F0030343605368C7
:102E100003F0F0038360536803F4E063C360526817
:102E20004FF4E06303EAD20202610448006800F054
:102E300007000860704700000010024000200240B8
:102E40000448054900684968044AC1F30221515CFD
:102E5000C8407047880900200010024060B5000893
:102E60000448054900684968044AC1F3C221515C1D
:102E7000C8407047880900200010024060B5000873
:102E800012A085B00FC88DE80F0014A0144B006885
:102E900004905968134801F00C02042A10D0082A43
:102EA0000ED1C1F38342C9031DF802000AD5596847
:102EB00004AAC1F34041515C0A4A5043B0FBF1F00F
:102EC00005B0704708494843FAE7000002030405CB
:102ED000060708090A0B0C0D0E0F10100102000066
:102EE0000010024000127A0000093D002DE9F84F61
:102EF00004006FD02078BE4DC00747D06868C0F38B
:102F00008100012807D06868C0F38100022809D138
:102F10006868C00306D52868800337D56068002834
:102F2000E7D033E06068B0F5803F0BD010B1B0F56A
:102F3000A02F11D0286820F480302860286820F461
:102F4000802002E0286840F480302860606888B102
:102F5000FFF7FCFD064609E0286840F48020286061
:102F6000F0E7FFF7F3FD801B642873D8286880031F
:102F7000F7D50BE0FFF7EAFD064604E0FFF7E6FDB4
:102F8000801B6428F1D828688003F7D42078DFF804
:102F9000648280074FF0010A4FF0000939D5686854
:102FA00010F00C0F07D06868C0F38100022809D127
:102FB0006868C00306D42868800714D520690128F2
:102FC00008D110E02069B0B1C8F800A0FFF7BEFD3D
:102FD000064605E007E1FFF7B9FD801B0228C4D8CB
:102FE00028688007F7D52868616920F0F80040EA72
:102FF000C10028600DE0C8F80090FFF7A7FD064665
:1030000004E0FFF7A3FD801B022823D8286880076F
:10301000F7D4207800072CD57748A169D9B1C0F83A
:1030200000A0FFF793FD064604E0FFF78FFD801B2D
:1030300002280FD8686A8007F7D570484FF4FA5114
:103040000068B0FBF1F0009000BF0098411E0091B5
:10305000FAD20EE07CE0C0F80090FFF777FD06465C
:1030600004E0FFF773FD801B022871D8686A8007AF
:10307000F7D4207840075BD5E8690027C00008D462
:10308000E86940F08050E861E869012700F080506D
:1030900000905B480168C90511D40168834641F47A
:1030A00080710160FFF752FD064604E0FFF74EFD18
:1030B000801B64284CD8DBF80000C005F6D5E0681A
:1030C00001280AD008B1052813D0286A20F0010091
:1030D0002862286A20F0040002E0286A40F001001B
:1030E0002862E06841F2883B88B1FFF72FFD064671
:1030F00009E0286A40F004002862EEE7FFF726FDA9
:10310000811B59455BD8286A8007F7D50BE0FFF78C
:103110001DFD064604E0FFF719FD811B59454ED8F9
:10312000286A8007F7D41FB1E86920F08050E86171
:10313000E069A8B36968C1F38101022946D0022879
:10314000484606D0C8F86000FFF700FD044639E0A5
:1031500035E04746C8F86000FFF7F8FC064604E093
:10316000FFF7F4FC801B022829D828688001F7D4D7
:10317000206AB0F5803F05D16868A16820F400306E
:1031800008436860D4E908010843696821F47411B0
:1031900008436860C7F860A0FFF7D8FC044605E064
:1031A00023E0FFF7D3FC001B022808D82868800121
:1031B000F7D51AE0FFF7CAFC001B022802D903204A
:1031C000BDE8F88F28688001F4D40EE00128F7D01C
:1031D0006868226A00F48031914204D1616A00F487
:1031E0007010884201D00120EAE70020E8E70000E3
:1031F0000010024000004242800442428809002040
:10320000007000407047704770B590F83C20012A6C
:103210002CD0012580F83C50022280F83D20026825
:103220005368946823F070060B6833435360104B67
:1032300002689A420ED00F4B9A420BD0B2F1804FE7
:1032400008D00D4B9A4205D00C4B9A4202D00C4B41
:103250009A4204D1496824F080031943916080F8B0
:103260003D50002180F83C10084670BD022070BD22
:10327000002C0140003401400004004000080040E0
:10328000000C004010B5040003D094F83D0010B1CC
:1032900007E0012010BD002084F83C00204600F02B
:1032A0001FF8022084F83D00211D206804F0B6FEBE
:1032B000012084F8460084F83E0084F83F0084F83A
:1032C000400084F8410084F8420084F8430084F808
:1032D000440084F8450084F83D00002010BD000043
:1032E00008B500680B4A0C49904207D1886940F440
:1032F00000608861886900F4006009E0074A904234
:1033000007D1C86940F00400C861C86900F0040032
:10331000009008BD002C0140001002400008004051
:1033200090F83D10012901D001207047022180F85A
:103330003D100168CA6842F00102CA6000680E4987
:1033400088420ED00D4988420BD0B0F1804F08D092
:103350000B49884205D00B49884202D00A4988426D
:1033600004D1816801F00701062903D0016841F00A
:103370000101016000207047002C01400034014031
:103380000004004000080040000C004070B50446F6
:1033900090F83C00012817D0012584F83C50022009
:1033A00084F83D002068826822F0770222F47F4290
:1033B00082600868502830D00DDC20284DD005DC14
:1033C00098B310283BD148E0022070BD302844D08B
:1033D000402834D139E0602828D0702806D0B0F5D4
:1033E000805F2CD0B0F5005F29D10AE0CB68D1E92D
:1033F0000121206804F058FE2068816841F07701BF
:1034000009E0CB68D1E90121206804F04DFE206875
:10341000816841F48041816011E0CA684968206890
:1034200004F054FE5021206807E016E0CA6849689D
:10343000206804F05CFE6021206804F03FFE84F800
:103440003D50002084F83C0070BDCA68496820687F
:1034500004F03CFE40212068EFE722680146104658
:10346000EBE7704770B50446006801694FF000054E
:10347000C943890715D4C168C943890711D4E91E16
:10348000016101202077206880698007204602D0F2
:10349000FFF7E7FF04E000F098F8204600F096F808
:1034A000257720680169C943490717D4C168C94312
:1034B000490713D46FF004010161022020772068CE
:1034C000806910F4407F204602D0FFF7CAFF04E075
:1034D00000F07BF8204600F079F825772068016934
:1034E000C943090716D4C168C943090712D46FF04C
:1034F00008010161042020772068C0698007204608
:1035000002D0FFF7AEFF04E000F05FF8204600F0C5
:103510005DF8257720680169C943C90617D4C168D9
:10352000C943C90613D46FF0100101610820207748
:103530002068C06910F4407F204602D0FFF791FF59
:1035400004E000F042F8204600F040F825772068BB
:103550000169C943C90708D1C168C943C90704D172
:10356000891E0161204600F033F820680169C943D3
:10357000090609D4C168C943090605D46FF0800162
:1035800001612046FFF73EFE20680169C9434906F4
:1035900009D4C168C943490605D46FF040010161EF
:1035A000204600F01FF820680169C94389060BD442
:1035B000C168C943890607D46FF020010161204624
:1035C000BDE87040FFF71FBE70BD70477047000038
:1035D00000680349884201D1FFF7BEBA7047000076
:1035E00000340140704710B504460068416994F802
:1035F0003920C1F3C011212A0BD151B1416921F009
:1036000080014161206B08B1FEF77AFE204604F08C
:1036100059FE2068416994F83A20C1F38011222AAA
:103620000BD151B1416921F040014161606B08B19A
:10363000FEF766FE204604F037FE002010BD7047FE
:1036400070B5026804461068D168536910F00F0F16
:1036500052D003F0010501F490762E435FD0C207EB
:1036600005D0CA0503D5E26B42F00102E2634207CE
:1036700005D5DA0703D0E26B42F00202E26382076B
:1036800005D5DA0703D0E26B42F00402E2630207D9
:1036900007D501F020022A4303D0E26B42F0080272
:1036A000E263E26B002A33D0800604D5880602D597
:1036B000204604F010FE20684069E16BC0F38010E2
:1036C000090700D428B3204604F0EEFD20684169C4
:1036D00049061AD5416921F040014161606BA0B1F2
:1036E0002D494163606BFEF72FFE002810D0606B00
:1036F000416BBDE870400847830610D58B060ED598
:103700002046BDE8704004F0E6BD2046FFF797FF75
:1037100070BD2046FFF793FF0020E06370BD0306F5
:103720002BD50B0629D594F839002128F6D1A068AD
:10373000B0F5805F01D12069B0B1206A411C2162DF
:10374000216800784860E08C401E0004000CE08492
:10375000E4D12068C16821F08001C1602068C1689F
:1037600041F04001C16070BD206A0088C0F30800CC
:103770005060206A801C2062E5E74006F3D54806C9
:10378000F1D5D168204621F04001D160202184F894
:10379000391000F0EFF970BD0982000870B504001F
:1037A00004D094F83900002510B106E0012070BD66
:1037B00084F83850204600F023F8242084F839009B
:1037C0002068C16821F40051C160204604F0CAFDA0
:1037D0002068016921F4904101612068416921F06C
:1037E0002A0141612068C16841F40051C160E5636C
:1037F000202084F8390084F83A00002070BD0000D1
:103800002DE9F04F85B000250095019502950395AF
:103810000446774E01687748022203234FF00408DC
:10382000B14229D1C16941F48011C161C16901F47A
:1038300080110491816941F010018161816901F079
:1038400010010491816941F020018161806969461C
:1038500000F020000490D002CDE9000203936648F6
:10386000FFF76AF8CDE90085694664480295FFF7DD
:1038700063F805B0BDE8F08FDFF884C1614F8026A2
:103880004FF480694FF0200A4FF4005B614544D14A
:10389000816941F480418161816901F48041049131
:1038A000816941F0040181618069694600F004008A
:1038B0000490B000CDE9000203933846FFF73CF8CE
:1038C000CDE90095694638460295FFF735F84F4F28
:1038D0004D4807F11401C7E90005C7E902563D61EB
:1038E00081E8200C3846FEF7EBFE08B1FDF738FD05
:1038F00067637C624448464F143801C7102061C793
:10390000434847F810597D61BD61FD61FEF7D8FE5F
:1039100008B1FDF725FD276333E0DFF8F8C0614506
:1039200031D1C16941F40031C161C16901F4003193
:103930000491816941F0040181618069694600F068
:103940000400CDE90330CDE900823846FEF7F4FFEC
:103950000820CDE90005694638460295FEF7ECFFE0
:103960002D4F294807F114011430C7E90005C7E9B4
:1039700002563D6181E8200C384633E0FDF7F0FC4B
:1039800034E07C6275E7254FB942FBD1C16941F44F
:103990008021C161C16901F480210491816941F0F4
:1039A0000801816180691E4F00F00800CDE90330F5
:1039B000CDE9009269463846FEF7BEFFF814CDE91E
:1039C0000005694638460295FEF7B6FF0E48154FCA
:1039D0002838C7E90005C7E902563D617D61BD6130
:1039E0003846FD61FEF76CFE0028C7D16763C8E763
:1039F000005000400010024000100140001401403F
:103A0000003801400008014058000240940F002097
:103A1000EC260020004400403027002000480040F1
:103A2000000C01407427002037B5044690F83A0096
:103A300082B0134620283AD1039AAAB3A3B394F8CC
:103A40003800012833D0012084F83800A262A38511
:103A50000025E563222084F83A00616B15488862EE
:103A6000616B1548C862616B14480863606B4563FD
:103A70002168606B091DFEF761FE206801684168DE
:103A8000009184F83850C16841F48071C1602068A9
:103A9000416941F0010141612068416941F0400103
:103AA0004161002005B030BDFFE70120FAE70220A8
:103AB000F8E70000638200089F820008198200086E
:103AC000704770472DE9F843044690F839001F46C7
:103AD00015460E4620284BD1C6B1BDB194F838002A
:103AE000012845D0012084F838004FF00008C4F8C0
:103AF0003C80212084F83900FFF728F8A58481460E
:103B0000E584A068B0F5805F03D004E00120BDE843
:103B1000F883206920B13546002684F838800EE00D
:103B20000025FAE78021204604F078FCA0B9ADB169
:103B300015F8010B21684860E08C401EE084E08CA1
:103B40004B464FF0000200970028EBD14FF04001A8
:103B5000204604F063FC30B10320D8E736F8020BAE
:103B6000C0F30800E6E7202084F839000020CEE703
:103B70000220CCE770470000134810B5418811B906
:103B8000017D062901D0002010BD01210E4C41808D
:103B9000463C807F2070062060700020A070A52029
:103BA000E07020716071A071E07120726072A0728B
:103BB000E072207360730E21204600F0F3F8010AD2
:103BC000A173E073012010BD623200202DE9F041A5
:103BD0008AB006462B4D2C4C28216846FCF73FFB4B
:103BE00000206F4605E02118497F27F81010401C7F
:103BF000C0B2217E8142F6D8207DDFF89080062871
:103C000004D1012241463846FDF744FC01224146D9
:103C10006846FDF731FCBDF800003074BDF80000C7
:103C2000052800D2E880207DDFF86480062804D1D2
:103C300008224146B81CFDF72DFC08224146B81C5D
:103C4000FDF71AFC002013E007EB4002231851880F
:103C50009B7F994202D0237D062B10D0082905D2E4
:103C600005EB40039984917832185174401CC0B21E
:103C7000217E8142E8D801200AB0BDE8F081002011
:103C8000FAE70000203100206232002030F00708FF
:103C900040E00708144810B5418811B9017D062994
:103CA00001D0002010BD104C01214180463C817F95
:103CB0002170062161701021A17090F82000E07041
:103CC000A52020716071A071E07120726072A072F5
:103CD000E072207360730E21204600F063F8010A41
:103CE000A173E073012010BD62320020144810B5AA
:103CF000418811B9017D062901D0002010BD104C6A
:103D000001214180463C817F217006216170122192
:103D1000A17090F82000E070A52020716071A07162
:103D2000E07120726072A072E072207360730E21E5
:103D3000204600F037F8010AA173E073012010BD9E
:103D400062320020154810B5418811B9017D06295D
:103D500001D0002010BD114C01214180463C817FE3
:103D60002170062161701421A170C17FE17090F86B
:103D700020002071A5206071A071E0712072607236
:103D8000A072E072207360730E21204600F00AF8E2
:103D9000010AA173E073012010BD0000623200200F
:103DA000FEE7000070B5094DFF22134605F5807649
:103DB00005E010F8014B54402A5D5A40335D491E1E
:103DC00089B2F6D203EB022080B270BD70AE00085B
:103DD000002203E0491E00F8012B89B20029F9D125
:103DE00070470000F0B58BB00546344C344E2821A6
:103DF0006846FCF734FAB4F81D00324F40BAADF80B
:103E00000000B4F81F0040BAADF80200B4F8210079
:103E100040BAADF80400B4F8230040BAADF806008B
:103E2000207D062804D1042239466846FDF732FB7E
:103E3000042239466846FDF71FFBBDF80000000A62
:103E40002874BDF80010CBB26B74BDF80210090ADB
:103E5000A974BDF80210E974BDF80410090A2975A7
:103E6000BDF804106975BDF80610090AA975BDF8FA
:103E70000810E975617F884205D1A27F934202D183
:103E8000207D062802D000200BB0F0BD0E48C17086
:103E9000827014F81F1F4170617801700168F1642D
:103EA00000BFA178C170E17881702179417061799A
:103EB00001700068706700BF0120E5E762320020F2
:103EC0001839002000C007081C030020F0B58BB093
:103ED00005461C4E1C4C28216846FCF7C0F9B4F876
:103EE0001D001A4F40BAADF80000207D062804D10D
:103EF000012239466846FDF7CDFA01223946684667
:103F0000FDF7BAFABDF80000000A2874BDF80000F9
:103F10006874BDF80000A0F57F41FF3901D0A6F814
:103F20006400287C617F884206D1687CA17F88423A
:103F300002D1207D062802D000200BB0F0BD012068
:103F4000FBE70000203100206232002040F007082B
:103F500070B5017845780846FCF762F93038C4B28C
:103F6000092C01D9E41FE4B22846FCF759F930388E
:103F7000C0B2092801D9C01FC0B200EB0410C0B202
:103F800070BD00002DE9F04F85B000243B4800943F
:103F9000019402940394816941F020018161816957
:103FA00001F020010491816941F00401816181697E
:103FB00001F004010491816941F008018161816986
:103FC00001F008010491816941F01001816180696B
:103FD000DFF8AC9000F01000049000221321484656
:103FE000FEF7AFFDDFF89CA04FF4405700223946A2
:103FF0005046FEF7A6FDDFF890B04FF4806800222F
:1040000041465846FEF79DFD132001250226CDE9C5
:104010000005CDE9024669464846FEF78DFC00974B
:104020000396CDE9015469465046FEF785FCB80079
:10403000CDE90004694650460294FEF77DFC4FF43A
:104040007070CDE90004694658460294FEF774FC8E
:104050004FF41060CDE90004694648460294FEF72B
:104060006BFCCDF800800396CDE9015469465846B3
:10407000FEF762FC05B0BDE8F08F000000100240C2
:1040800000080140000C01400010014010B5002262
:1040900005212720FEF7E6FD2720FEF7D5FD0022AB
:1040A00005212520FEF7DEFD2520FEF7CDFD0022AF
:1040B00005212620FEF7D6FD2620FEF7C5FD0022AD
:1040C00005211E20FEF7CEFD1E20FEF7BDFD0022BD
:1040D00005211920FEF7C6FD1920FEF7B5FD0022C7
:1040E00005211020FEF7BEFD1020FEF7ADFD0022D9
:1040F00005210F20FEF7B6FD0F20FEF7A5FD0022DB
:1041000005210D20FEF7AEFDBDE810400D20FEF7A5
:104110009BBD000010B586B000241848009401949F
:1041200002940394049414490594C0E900144FF6D2
:10413000FF71C0E902414FF40071C0E904148461C9
:10414000FFF7A0F808B172B6FEE74FF48050009078
:1041500069460A48FFF71AF908B172B6FEE70494F7
:1041600004A906480594FFF74FF8002801D072B65D
:10417000FEE706B010BD0000002C01405C240020CA
:1041800010B586B00024164800940194029403945C
:10419000049412490594C0E900144FF6FF71C0E978
:1041A000024104618461FFF76DF808B172B6FEE761
:1041B0004FF48050009069460948FFF7E7F808B1CE
:1041C00072B6FEE7049404A905480594FFF71CF8AD
:1041D000002801D072B6FEE706B010BD000800400E
:1041E000A424002010B5114C0F480C2120604FF47E
:1041F000165060600020A060E060C4E90401A06186
:10420000E0612046FFF7CAFA08B172B6FEE72068FF
:10421000C16841F01001C160BDE810404FF48072E8
:1042200003490248FFF700BC003801402C2500205C
:10423000100D002010B5114C0F480C2120604FF4D8
:10424000164060600020A060E060C4E90401A06145
:10425000E0612046FFF7A2FA08B172B6FEE72068D7
:10426000C16841F01001C160BDE810404FF4807298
:1042700003490248FFF7D8BB004400406C250020EA
:104280000021002010B5114C0F480C2120604FF484
:10429000165060600020A060E060C4E90401A061E5
:1042A000E0612046FFF77AFA08B172B6FEE72068AF
:1042B000C16841F01001C160BDE810404FF4807248
:1042C00003490248FFF7B0BB00480040AC2500207E
:1042D000100E0020FEE7FEE72DE9F0412B4F8AB0DB
:1042E000A7F58C66A6F59064002508222849684643
:1042F000FDF7C2F869464FF6FF7808E031F815007F
:10430000404502D007EB450290866D1CEDB238881F
:10431000A842F3D801221F496846FDF7ADF8BDF861
:1043200000004546A84200D038811A4901223831A0
:104330006846FDF7A1F8BDF80000A84201D14FF48E
:104340001670A6F84200A6F888000023A6F8CE0052
:1043500098465E1EA4F80080E680A6806580402115
:1043600004F10800FFF734FD5B1CDBB24834082B76
:10437000F0D300200222084B398802E0401C1A705A
:10438000C0B28142FAD80AB0BDE8F08120310020E5
:1043900020E0070820F0070814030020F0B585B0DE
:1043A0000546184E184C14216846FBF758FFB4F820
:1043B0001D00164F40BAADF80000207D062804D13C
:1043C000012239466846FDF765F80020ADF8000087
:1043D000012239466846FDF74FF8BDF80010A6F8EF
:1043E0004210090A2974BDF80000C0B26874627FE7
:1043F000914205D1A17F884202D1012005B0F0BDD4
:104400000020FBE7C02C00206232002058F0070893
:104410002DE9F0418AB006462B4D2C4C28216846E8
:10442000FBF71DFF00206F4605E02118497F27F8A4
:104430001010401CC0B2217E8142F6D8207DDFF8EA
:104440009080062804D1012241463846FDF722F823
:10445000012241466846FDF70FF8BDF800003074B0
:10446000BDF80000052800D22881207DDFF8648097
:10447000062804D108224146B81CFDF70BF8082293
:104480004146B81CFCF7F8FF002013E007EB4002A0
:10449000231851889B7F994202D0237D062B10D090
:1044A000082905D205EB400399869178321851749A
:1044B000401CC0B2217E8142E8D801200AB0BDE88C
:1044C000F0810020FAE70000203100206232002055
:1044D00020F0070820E007087CB51748002100916C
:1044E0000191028812B9027D062A01D000207CBD0C
:1044F0000122114C0280D23C807F2070062565701D
:10450000A1701022E2702171FF2363718DF8000009
:104510008DF801508DF802108DF804108DF80320ED
:104520008DF8053029466846FFF73CFC010AA17169
:10453000E07101207CBD0000623200202DE9F041D5
:10454000754A04467248917F724B744D4E1E082E78
:1045500002D30020BDE8F0812026E672927F6274CB
:1045600003EBC1160022B6F87A7047234FF07F0C98
:104570004FF0FF0E97B1A37484F813C084F814E0D1
:104580006275A37584F817C084F818E06276A37684
:1045900084F81BC084F81CE0627729E0B6F900704B
:1045A0003F0EA774B6F900703F0CE77437883F0AD6
:1045B000277537786775B6F928703F0EA775B6F975
:1045C00028703F0CE775378D3F0A277696F82870DC
:1045D0006776B6F950703F0EA776B6F950703F0C6B
:1045E000E776B6F850703F0A277796F850606677FE
:1045F000B0F87A60BEB1A37784F81FC084F820E0D9
:1046000084F8212084F8223084F823C084F824E040
:1046100084F8252084F8263084F827C084F828E020
:1046200084F8292033E0B0F90060360EA677B0F99F
:104630000060360CE6770688360A84F8206010F8A9
:10464000286B84F8216030F9286B360E84F82260DC
:1046500030F9286C360C84F8236030F8286C360A60
:1046600084F8246010F8286C84F82560B0F90060A4
:10467000360E84F82660B0F90060360C84F82760A6
:104680000688360A84F82860007884F8290001EB4F
:10469000810705EBC706F08B68B104F82A3F84F860
:1046A00001C084F802E0E270237184F805C084F848
:1046B00006E0E2712AE055F83700FBF78CFF000EA8
:1046C00004F82A0F55F83700FBF785FF000C6070DF
:1046D00055F83700FBF77FFF000AA07055F8370048
:1046E000FBF779FFE070B069FBF775FF000E2071F2
:1046F000B069FBF770FF000C6071B069FBF76BFFEE
:10470000000AA071B069FBF766FFE071012021E7A4
:10471000983B00201C3C0020623200201839002009
:104720002DE9FE4F0446E1480290E4480190E44838
:10473000012700900020DFF87093DFF874B3DD4BA1
:10474000DFF874A30146064605468646A7F1010C2C
:104750000FE00AEB4002401C92F82480C0B24144B2
:1047600092F8148092F8342046442A44C9B2F6B232
:10477000D5B26045EDDB0020724604EB000C401C16
:10478000C0B28CF810200428F7D307EBC70000EB69
:10479000471C0BEB4C0C9CF8020004F8140F002093
:1047A0006070A070E0709CF840202271607107EB8F
:1047B0008702A07102EB871CE07113F81C202272A3
:1047C0006072A07203EB4C02E07292F8288084F8C9
:1047D0000C806073A073E07313F81C302374607452
:1047E000A0749246E07492F8282022756075A07536
:1047F000E07501EBC10000EB41120BEB42004FF002
:104800000308B0F89E00143C10B184F82C8005E039
:10481000491CC8B2FDF702FC84F82C0006EB061018
:1048200000EB4001009800EB4100B0F8C41011B15A
:1048300084F8308003E090F8BE1084F83010C5EBA7
:10484000C50101EB8102019901EB4201B1F8802021
:104850001AB1414684F8348004E011F87A2F84F8C4
:104860003420897884F83810B0F8C41011B184F875
:104870003C8003E090F8C00084F83C00002604F877
:104880002D6F6670A67026716671A67126726672AB
:10489000A67226736673A67326746674A6749AF855
:1048A0002800E07426756675A6759AF82800E075EC
:1048B00026766676A67600202D3C2118401CC0B2D4
:1048C00081F848602028F8D3029807EB870100EBB5
:1048D000C105E88B40B184F8686084F8696084F8A9
:1048E0006A6084F86B600BE0686884F86800010A0D
:1048F00084F86910010C84F86A10000E84F86B00CB
:10490000E88BDFF8C08140B184F86C6084F86D609A
:1049100084F86E6084F86F6013E009EBC710B0F99B
:104920002A00FBF74AFE4146FBF7FCFC84F86C00CA
:10493000010A84F86D10010C84F86E10000E84F8E2
:104940006F00E88B40B184F8706084F8716084F87F
:10495000726084F8736013E009EBC710B0F90200CD
:10496000FBF72BFE4146FBF7DDFC84F87000010AE3
:1049700084F87110010C84F87210000E84F8730032
:10498000E88B40B184F8746084F8756084F87660D0
:1049900084F8776013E009EBC710B0F92A00FBF741
:1049A0000CFE4146FBF7BEFC84F87400010A84F853
:1049B0007510010C84F87610000E84F87700E88BEF
:1049C00040B184F8786084F8796084F87A6084F87B
:1049D0007B6013E009EBC710B0F95200FBF7EDFD67
:1049E0004146FBF79FFC84F87800010A84F87910AF
:1049F000010C84F87A10000E84F87B00E88B58B123
:104A0000762084F87C007F2084F87D00FF2084F8E5
:104A10007E0084F87F600BE0A86984F87C00010ABE
:104A200084F87D10010C84F87E10000E84F87F005D
:104A3000E88B84F8806084F8816084F8826084F870
:104A40008360E88B84F8846084F8856084F88660ED
:104A500084F88760E88B84F8886084F8896084F83B
:104A60008A6084F88B60E88B40B184F88C6084F8AD
:104A70008D6084F88E6084F88F600BE0A86984F8FC
:104A80008C00010A84F88D10010C84F88E10000E41
:104A900084F88F00E88B04F8906F01206670A67090
:104AA000E670BDE8FE8F00001C3C00201839002095
:104AB0001C4400203C49002020310020C02C002054
:104AC000B6320020CDCCCC3D2DE9F043DFF8149375
:104AD0000021A5224318491CC9B21A740829F9D922
:104AE00000210B4600EB8102491C13765376937626
:104AF000C9B2D3760829F5D9012176267F274FF050
:104B0000FF0C01EB810409EBC402D58B55B101EB1D
:104B1000410404EBC10400EB840423736373A373A7
:104B2000E37312E001EB410505EBC10559F8344090
:104B300000EB85054FEA14282C7385F80D804FEAA9
:104B4000144885F80E80240EEC73D48B54B101EB1D
:104B5000410404EBC10400EB840423746374A37464
:104B6000E37411E001EB410505EBC10500EB8505A0
:104B700094682C744FEA142885F811804FEA144881
:104B800085F81280240EEC74D48B54B101EB4104EF
:104B900004EBC10400EB840423756375A375E3750E
:104BA00011E001EB410505EBC10500EB8505D4687B
:104BB0002C754FEA142885F815804FEA144885F8BB
:104BC0001680240EEC75D48B54B101EB410404EB38
:104BD000C10400EB840423766376A376E37611E0C8
:104BE00001EB410505EBC10500EB850514692C7649
:104BF0004FEA142885F819804FEA144885F81A807E
:104C0000240EEC76D48B54B101EB410404EBC104C7
:104C100000EB840423776377A377E37711E001EB5C
:104C2000410505EBC10500EB850554692C774FEA7A
:104C3000142885F81D804FEA144885F81E80240E3C
:104C4000EC77D48B64B101EB410404EBC10400EBBD
:104C5000840404F8206F677084F802C0E37012E0E7
:104C600001EB410505EBC10500EB8505946905F8ED
:104C7000204F4FEA142885F801804FEA144885F840
:104C80000280240EEC70D48B64B101EB410404EB80
:104C9000C10400EB840404F8246F677084F802C038
:104CA000E37012E001EB410505EBC10500EB850562
:104CB000946905F8244F4FEA142885F801804FEADB
:104CC000144885F80280240EEC70D48B64B101EB9B
:104CD000410404EBC10400EB840404F8286F6770FE
:104CE00084F802C0E37012E001EB410505EBC10559
:104CF00000EB8505946905F8284F4FEA142885F8DC
:104D000001804FEA144885F80280240EEC70D48BA1
:104D100064B101EB410404EBC10400EB840404F82A
:104D20002C6F677084F802C0E37012E001EB41055C
:104D300005EBC10500EB8505946905F82C4F4FEA9A
:104D4000142885F801804FEA144885F80280240E63
:104D5000EC70D48B64B101EB410404EBC10400EBB3
:104D6000840404F8306F677084F802C0E37012E0C6
:104D700001EB410505EBC10500EB8505946905F8DC
:104D8000304F4FEA142885F801804FEA144885F81F
:104D90000280240EEC70D48B64B101EB410202EB73
:104DA000C10200EB820202F8346F577082F802C031
:104DB000D3700EE001EB410404EBC10400EB84046A
:104DC000926904F8342F150A6570150CA570120E3F
:104DD000E270491CC9B204297FF693AE0120BDE8F8
:104DE000F0830000183900202DE9FE4F0446D94811
:104DF0000290DC480190DC48022700900020DFF898
:104E00005093DFF854B3D54BDFF854A30146064660
:104E10000546A7F1010C0FE00AEB4002401C92F896
:104E20002480C0B2414492F8148092F83420464461
:104E30002A44C9B2F6B2D5B26045EDDB0020024685
:104E400004EB000C401CC0B28CF810200428F7D3EF
:104E500007EBC70000EB471C0BEB4C0C9CF8020067
:104E600004F8140F00206070A070E0709CF84020DF
:104E70002271607107EB8702A07102EB871CE07161
:104E800013F81C2022726072A07203EB4C02E072D5
:104E900092F8288084F80C806073A073E07313F894
:104EA0001C3023746074A0749246E07492F8282039
:104EB00022756075A075E07501EBC10000EB411231
:104EC0000BEB42004FF00308B0F89E00143C10B109
:104ED00084F82C8005E0491CC8B2FDF79FF884F8DF
:104EE0002C0006EB061000EB4001009800EB41009F
:104EF000B0F8C41011B184F8308003E090F8BE100F
:104F000084F83010C5EBC50101EB8102019901EB7A
:104F10004201B1F880201AB1414684F8348004E09F
:104F200011F87A2F84F83420897884F83810B0F892
:104F3000C41011B184F83C8003E090F8C00084F8FC
:104F40003C00002604F82D6F6670A670267166710D
:104F5000A67126726672A67226736673A67326748D
:104F60006674A6749AF82800E07426756675A675AE
:104F70009AF82800E07526766676A67600202D3C05
:104F80002118401CC0B281F848602028F8D302984C
:104F900007EB870100EBC105E88B40B184F868603E
:104FA00084F8696084F86A6084F86B600BE0686874
:104FB00084F86800010A84F86910010C84F86A100A
:104FC000000E84F86B00E88BDFF8A08140B184F814
:104FD0006C6084F86D6084F86E6084F86F6013E034
:104FE00009EBC710B0F92A00FBF7E7FA4146FBF7D7
:104FF00099F984F86C00010A84F86D10010C84F8AA
:105000006E10000E84F86F00E88B40B184F8706079
:1050100084F8716084F8726084F8736013E009EBBF
:10502000C710B0F90200FBF7C8FA4146FBF77AF95E
:1050300084F87000010A84F87110010C84F8721071
:10504000000E84F87300E88B40B184F8746084F833
:10505000756084F8766084F8776013E009EBC71018
:10506000B0F92A00FBF7A9FA4146FBF75BF984F88F
:105070007400010A84F87510010C84F87610000E93
:1050800084F87700E88B40B184F8786084F8796020
:1050900084F87A6084F87B6013E009EBC710B0F9FC
:1050A0005200FBF78AFA4146FBF73CF984F8780096
:1050B000010A84F87910010C84F87A10000E84F843
:1050C0007B00E88B58B1762084F87C007F2084F840
:1050D0007D00FF2084F87E0084F87F600BE0A869E3
:1050E00084F87C00010A84F87D10010C84F87E109D
:1050F000000E84F87F00E88B84F8806084F881607B
:1051000084F8826084F88360E88B84F8846084F893
:10511000856084F8866084F88760E88B84F888600E
:1051200084F8896084F88A6084F88B60E88B84F85E
:105130008C6084F88D6084F88E6084F88F60E88BD2
:1051400004F8906F01206670A670E670BDE8FE8FCF
:105150001C3C0020183900201C4400203C49002041
:1051600020310020C02C0020B6320020CDCCCC3D18
:10517000F0B503269C4D9D4C9D4B0022114687188F
:10518000521CD2B23974042AF9D306EBC60202EBE0
:10519000461204EB4202947800F8144F417081707B
:1051A000C17092F840200271417106EB8602817154
:1051B00002EB8614C17113F81420027241728172DD
:1051C00003EB4402C17212F8287F077341738173A5
:1051D000C17313F81470077441748174C174177823
:1051E000077541758175C17513F81470077641769E
:1051F0008176C1761778077741778177C17713F881
:10520000143080F8203080F8211080F8221080F8C7
:105210002310137880F8243080F8251080F82610A9
:1052200080F82710137880F8283080F8291080F84B
:105230002A1080F82B10137880F82C3080F82D106D
:1052400080F82E1080F82F10127880F8302080F827
:10525000311080F8321080F833100022143883188F
:10526000521CD2B283F84810202AF8D306EB8603EA
:1052700005EBC302D48B44B180F8681080F8691044
:1052800080F86A1080F86B100CE055F8333080F825
:1052900068301C0A80F869401C0C80F86A401B0EBC
:1052A00080F86B30D38B43B180F86C1080F86D10B0
:1052B00080F86E1080F86F100BE0936880F86C3007
:1052C0001C0A80F86D401C0C80F86E401B0E80F8A4
:1052D0006F30D38B43B180F8701080F8711080F874
:1052E000721080F873100BE0D36880F870301C0ADD
:1052F00080F871401C0C80F872401B0E80F87330EF
:10530000D38B43B180F8741080F8751080F8761054
:1053100080F877100BE0136980F874301C0A80F86D
:1053200075401C0C80F876401B0E80F87730D38BCC
:1053300043B180F8781080F8791080F87A1080F8FE
:105340007B100BE0536980F878301C0A80F87940B4
:105350001C0C80F87A401B0E80F87B30D38B5BB13D
:10536000762380F87C307F2380F87D30FF2380F81F
:105370007E3080F87F100BE0936980F87C301C0A47
:1053800080F87D401C0C80F87E401B0E80F87F303A
:10539000D38B80F8801080F8811080F8821080F81C
:1053A0008310D38B80F8841080F8851080F88610E5
:1053B00080F88710D38B80F8881080F8891080F8E7
:1053C0008A1080F88B10D38B80F88C1080F88D10A9
:1053D00080F88E1080F88F10D28B00F8901F4170EB
:1053E0008170C1700120F0BD183900201C440020DC
:1053F0003C490020F0B504269C4D9D4C9D4B00225D
:1054000011468718521CD2B23974042AF9D306EB1C
:10541000C60202EB461204EB4202947800F8144FE5
:1054200041708170C17092F840200271417106EBA9
:105430008602817102EB8614C17113F81420027286
:105440004172817203EB4402C17212F8287F077324
:1054500041738173C17313F81470077441748174BC
:10546000C1741778077541758175C17513F814708B
:10547000077641768176C17617780777417781770D
:10548000C17713F8143080F8203080F8211080F8AC
:10549000221080F82310137880F8243080F825102B
:1054A00080F8261080F82710137880F8283080F8CC
:1054B000291080F82A1080F82B10137880F82C30EF
:1054C00080F82D1080F82E1080F82F10127880F8B8
:1054D000302080F8311080F8321080F8331000222C
:1054E00014388318521CD2B283F84810202AF8D3FB
:1054F00006EB860305EBC302D48B44B180F8681039
:1055000080F8691080F86A1080F86B100CE055F88C
:10551000333080F868301C0A80F869401C0C80F831
:105520006A401B0E80F86B30D38B43B180F86C104F
:1055300080F86D1080F86E1080F86F100BE09368A3
:1055400080F86C301C0A80F86D401C0C80F86E40AE
:105550001B0E80F86F30D38B43B180F8701080F849
:10556000711080F8721080F873100BE0D36880F827
:1055700070301C0A80F871401C0C80F872401B0EC1
:1055800080F87330D38B43B180F8741080F87510B5
:1055900080F8761080F877100BE0136980F874308B
:1055A0001C0A80F875401C0C80F876401B0E80F8B1
:1055B0007730D38B43B180F8781080F8791080F879
:1055C0007A1080F87B100BE0536980F878301C0A61
:1055D00080F879401C0C80F87A401B0E80F87B30F4
:1055E000D38B5BB1762380F87C307F2380F87D30CD
:1055F000FF2380F87E3080F87F100BE0936980F8FD
:105600007C301C0A80F87D401C0C80F87E401B0E0C
:1056100080F87F30D38B80F8801080F8811080F87C
:10562000821080F88310D38B80F8841080F8851066
:1056300080F8861080F88710D38B80F8881080F867
:10564000891080F88A1080F88B10D38B80F88C102A
:1056500080F88D1080F88E1080F88F10D28B00F8B3
:10566000901F41708170C1700120F0BD1839002079
:105670001C4400203C490020F0B505269C4D9D4C63
:105680009D4B002211468718521CD2B23974042A4D
:10569000F9D306EBC60202EB461204EB4202947801
:1056A00000F8144F41708170C17092F8402002716F
:1056B000417106EB8602817102EB8614C17113F809
:1056C000142002724172817203EB4402C17212F81B
:1056D000287F077341738173C17313F814700774C3
:1056E00041748174C1741778077541758175C175EE
:1056F00013F81470077641768176C17617780777AC
:1057000041778177C17713F8143080F8203080F822
:10571000211080F8221080F82310137880F82430AC
:1057200080F8251080F8261080F82710137880F86C
:10573000283080F8291080F82A1080F82B10137870
:1057400080F82C3080F82D1080F82E1080F82F1063
:10575000127880F8302080F8311080F8321080F80C
:105760003310002214388318521CD2B283F8481028
:10577000202AF8D306EB860305EBC302D48B44B191
:1057800080F8681080F8691080F86A1080F86B1053
:105790000CE055F8333080F868301C0A80F8694016
:1057A0001C0C80F86A401B0E80F86B30D38B43B121
:1057B00080F86C1080F86D1080F86E1080F86F1013
:1057C0000BE0936880F86C301C0A80F86D401C0C6C
:1057D00080F86E401B0E80F86F30D38B43B180F899
:1057E000701080F8711080F8721080F873100BE060
:1057F000D36880F870301C0A80F871401C0C80F867
:1058000072401B0E80F87330D38B43B180F8741054
:1058100080F8751080F8761080F877100BE0136927
:1058200080F874301C0A80F875401C0C80F87640B3
:105830001B0E80F87730D38B43B180F8781080F856
:10584000791080F87A1080F87B100BE0536980F8AB
:1058500078301C0A80F879401C0C80F87A401B0EC6
:1058600080F87B30D38B5BB1762380F87C307F234C
:1058700080F87D30FF2380F87E3080F87F100BE0C9
:10588000936980F87C301C0A80F87D401C0C80F8FD
:105890007E401B0E80F87F30D38B80F8801080F81C
:1058A000811080F8821080F88310D38B80F88410E8
:1058B00080F8851080F8861080F88710D38B80F8E8
:1058C000881080F8891080F88A1080F88B10D38BAC
:1058D00080F88C1080F88D1080F88E1080F88F1072
:1058E000D28B00F8901F41708170C1700120F0BD13
:1058F000183900201C4400203C490020F0B5062641
:105900009C4D9D4C9D4B002211468718521CD2B2D3
:105910003974042AF9D306EBC60202EB461204EBF3
:105920004202947800F8144F41708170C17092F86F
:1059300040200271417106EB8602817102EB8614F0
:10594000C17113F8142002724172817203EB440298
:10595000C17212F8287F077341738173C17313F802
:105960001470077441748174C17417780775417598
:105970008175C17513F81470077641768176C1760A
:105980001778077741778177C17713F8143080F85B
:10599000203080F8211080F8221080F8231013782E
:1059A00080F8243080F8251080F8261080F8271021
:1059B000137880F8283080F8291080F82A1080F8B1
:1059C0002B10137880F82C3080F82D1080F82E10D2
:1059D00080F82F10127880F8302080F8311080F88D
:1059E000321080F83310002214388318521CD2B2BF
:1059F00083F84810202AF8D306EB860305EBC30290
:105A0000D48B44B180F8681080F8691080F86A106F
:105A100080F86B100CE055F8333080F868301C0AC1
:105A200080F869401C0C80F86A401B0E80F86B30CF
:105A3000D38B43B180F86C1080F86D1080F86E1035
:105A400080F86F100BE0936880F86C301C0A80F8C7
:105A50006D401C0C80F86E401B0E80F86F30D38BAD
:105A600043B180F8701080F8711080F8721080F8DF
:105A700073100BE0D36880F870301C0A80F8714016
:105A80001C0C80F872401B0E80F87330D38B43B12E
:105A900080F8741080F8751080F8761080F8771010
:105AA0000BE0136980F874301C0A80F875401C0CF8
:105AB00080F876401B0E80F87730D38B43B180F8A6
:105AC000781080F8791080F87A1080F87B100BE05D
:105AD000536980F878301C0A80F879401C0C80F8F3
:105AE0007A401B0E80F87B30D38B5BB1762380F835
:105AF0007C307F2380F87D30FF2380F87E3080F873
:105B00007F100BE0936980F87C301C0A80F87D40A0
:105B10001C0C80F87E401B0E80F87F30D38B80F801
:105B2000801080F8811080F8821080F88310D38B69
:105B300080F8841080F8851080F8861080F887102F
:105B4000D38B80F8881080F8891080F88A1080F84C
:105B50008B10D38B80F88C1080F88D1080F88E100D
:105B600080F88F10D28B00F8901F41708170C17047
:105B70000120F0BD183900201C4400203C490020C1
:105B8000F0B507269C4D9D4C9D4B00221146871871
:105B9000521CD2B23974042AF9D306EBC60202EBC6
:105BA000461204EB4202947800F8144F4170817061
:105BB000C17092F840200271417106EB860281713A
:105BC00002EB8614C17113F81420027241728172C3
:105BD00003EB4402C17212F8287F0773417381738B
:105BE000C17313F81470077441748174C174177809
:105BF000077541758175C17513F814700776417684
:105C00008176C1761778077741778177C17713F866
:105C1000143080F8203080F8211080F8221080F8AD
:105C20002310137880F8243080F8251080F826108F
:105C300080F82710137880F8283080F8291080F831
:105C40002A1080F82B10137880F82C3080F82D1053
:105C500080F82E1080F82F10127880F8302080F80D
:105C6000311080F8321080F8331000221438831875
:105C7000521CD2B283F84810202AF8D306EB8603D0
:105C800005EBC302D48B44B180F8681080F869102A
:105C900080F86A1080F86B100CE055F8333080F80B
:105CA00068301C0A80F869401C0C80F86A401B0EA2
:105CB00080F86B30D38B43B180F86C1080F86D1096
:105CC00080F86E1080F86F100BE0936880F86C30ED
:105CD0001C0A80F86D401C0C80F86E401B0E80F88A
:105CE0006F30D38B43B180F8701080F8711080F85A
:105CF000721080F873100BE0D36880F870301C0AC3
:105D000080F871401C0C80F872401B0E80F87330D4
:105D1000D38B43B180F8741080F8751080F876103A
:105D200080F877100BE0136980F874301C0A80F853
:105D300075401C0C80F876401B0E80F87730D38BB2
:105D400043B180F8781080F8791080F87A1080F8E4
:105D50007B100BE0536980F878301C0A80F879409A
:105D60001C0C80F87A401B0E80F87B30D38B5BB123
:105D7000762380F87C307F2380F87D30FF2380F805
:105D80007E3080F87F100BE0936980F87C301C0A2D
:105D900080F87D401C0C80F87E401B0E80F87F3020
:105DA000D38B80F8801080F8811080F8821080F802
:105DB0008310D38B80F8841080F8851080F88610CB
:105DC00080F88710D38B80F8881080F8891080F8CD
:105DD0008A1080F88B10D38B80F88C1080F88D108F
:105DE00080F88E1080F88F10D28B00F8901F4170D1
:105DF0008170C1700120F0BD183900201C440020C2
:105E00003C490020F0B508269C4D9D4C9D4B00223E
:105E100011468718521CD2B23974042AF9D306EB02
:105E2000C60202EB461204EB4202947800F8144FCB
:105E300041708170C17092F840200271417106EB8F
:105E40008602817102EB8614C17113F8142002726C
:105E50004172817203EB4402C17212F8287F07730A
:105E600041738173C17313F81470077441748174A2
:105E7000C1741778077541758175C17513F8147071
:105E8000077641768176C1761778077741778177F3
:105E9000C17713F8143080F8203080F8211080F892
:105EA000221080F82310137880F8243080F8251011
:105EB00080F8261080F82710137880F8283080F8B2
:105EC000291080F82A1080F82B10137880F82C30D5
:105ED00080F82D1080F82E1080F82F10127880F89E
:105EE000302080F8311080F8321080F83310002212
:105EF00014388318521CD2B283F84810202AF8D3E1
:105F000006EB860305EBC302D48B44B180F868101E
:105F100080F8691080F86A1080F86B100CE055F872
:105F2000333080F868301C0A80F869401C0C80F817
:105F30006A401B0E80F86B30D38B43B180F86C1035
:105F400080F86D1080F86E1080F86F100BE0936889
:105F500080F86C301C0A80F86D401C0C80F86E4094
:105F60001B0E80F86F30D38B43B180F8701080F82F
:105F7000711080F8721080F873100BE0D36880F80D
:105F800070301C0A80F871401C0C80F872401B0EA7
:105F900080F87330D38B43B180F8741080F875109B
:105FA00080F8761080F877100BE0136980F8743071
:105FB0001C0A80F875401C0C80F876401B0E80F897
:105FC0007730D38B43B180F8781080F8791080F85F
:105FD0007A1080F87B100BE0536980F878301C0A47
:105FE00080F879401C0C80F87A401B0E80F87B30DA
:105FF000D38B5BB1762380F87C307F2380F87D30B3
:10600000FF2380F87E3080F87F100BE0936980F8E2
:106010007C301C0A80F87D401C0C80F87E401B0EF2
:1060200080F87F30D38B80F8801080F8811080F862
:10603000821080F88310D38B80F8841080F885104C
:1060400080F8861080F88710D38B80F8881080F84D
:10605000891080F88A1080F88B10D38B80F88C1010
:1060600080F88D1080F88E1080F88F10D28B00F899
:10607000901F41708170C1700120F0BD183900205F
:106080001C4400203C4900202DE9F04F87B0044615
:10609000C5480590C5480090C6480490C64803907E
:1060A000C34BC748002702909A7F0192DFF80CC3C8
:1060B000521E3D463E46BB463846082A1AD30020AB
:1060C00007B0BDE8F08F009901EB4001401C91F84A
:1060D0002480C0B2474491F81480FFB2454491F83F
:1060E0003480EDB2464491F84480F6B208EB0B01DF
:1060F00001F0FF0B9042E6DB2820E072987F60748D
:1061000007EBC70000EB47100CEB400A4FF0030908
:10611000BAF89E0010B184F8129004E0781CC0B266
:10612000FBF77CFFA07405EB051000EB4001039822
:1061300000EB4105B5F8C40010B184F8139002E0FB
:1061400095F8BE00E074FCF701FD9E490860C6EBBF
:10615000C60000EB8001049800EB4106B6F8800011
:1061600018B1484684F8149004E096F87A00207537
:1061700096F87C006075B5F8C40010B184F81690EC
:1061800002E095F8C000A0750BEB8B01059801EBC0
:106190008B1100EB4100B0F80E1111B184F817908B
:1061A00002E090F80801E07502984FF0A50B90F816
:1061B000F2002076BAF89E009AF87400607684F8AF
:1061C0001AB084F81BB0DDE9000100EB4108B8F813
:1061D000220001280BD9BAF8F00010B184F81C9005
:1061E00007E0B81CC0B2FBF719FF207701E084F884
:1061F0001CB0B8F81200012816D9B5F82A0110B160
:106200004846607704E095F82401607795F8260108
:1062100084F82000B8F83200012821D9B6F8C60069
:1062200020B14846A07706E05846EAE796F8C00055
:10623000A07796F8C200E07784F821B084F822B005
:1062400084F823B084F824B084F825B0B8F822008C
:1062500002280ED9BAF8420120B184F826900AE04B
:106260005846DFE7F81CC0B2FBF7D8FE84F82600DA
:1062700001E084F826B0B8F81200022819D9B5F860
:10628000900118B1484684F8270005E095F88A0186
:1062900084F8270095F88C0184F82A00B8F83200B9
:1062A000022824D9B6F80C0128B1484684F8280001
:1062B00007E05846E7E796F8060184F8280096F8C4
:1062C000080184F8290084F82BB084F82CB084F8F5
:1062D0002DB084F82EB084F82FB0B8F8220003282F
:1062E0000ED9BAF8940120B184F830900AE05846EB
:1062F000DCE73F1DF8B2FBF791FE84F8300001E0C7
:1063000084F830B0B8F81200032819D9B5F8F601AE
:1063100018B184F8319084F8349095F8F00184F83D
:10632000310095F8F20184F83400B8F832000428FE
:1063300037D9B6F8520138B1484684F8320009E03E
:10634000584684F831B0EEE796F84C0184F83200F4
:1063500096F84E0184F8330084F835B084F836B0EE
:1063600084F837B0174884F838B084F839B000683A
:10637000B0F5005F13D2002004F8140F6070A07015
:10638000E070A072E0722073607320756075A07574
:10639000E075A077E07784F8200084F821000120E0
:1063A0008EE65846C9E700003C4900202031002015
:1063B00062320020C02C0020B63200201C44002095
:1063C000DC510020180300202DE9F0416449044607
:1063D0006048897FDFF880C1604DA1F1510E002235
:1063E00047237F26FF27BEF10E0F24D2607C00EBEF
:1063F000800005EBC005A5F58055B5F89E0320B1DA
:10640000A374E67427756275A2E0D5F8800305F5DC
:106410006075FAF7E0F8000EA0742868FAF7DBF868
:10642000000CE0742868FAF7D6F8000A207528688E
:10643000FAF7D1F885E0A1F161050E2D3ED2607C1E
:106440000CEBC010A0F54050B0F87A1059B1A3740D
:10645000E67427756275A375E67527766276A3766E
:10646000E67627776277B0F90010090EA174B0F9CB
:106470000010090CE1740188090A21750178617521
:10648000B0F92810090EA175B0F92810090CE175B2
:10649000018D090A217690F828106176B0F9501024
:1064A000090EA176B0F95010090CE176B0F8501041
:1064B000090A217790F85000607749E0A1F1710551
:1064C0000E2D45D3103D0E2D42D3603D022D3AD204
:1064D000B0F87A1061B1A374E67427756275A3757C
:1064E000E67527766276A376E676277762772FE0E1
:1064F000B0F90010090EA174B0F90010090CE17494
:106500000188090A217501786175B0F92810090E12
:10651000A174B0F92810090CE174018D090A2175E4
:1065200090F828106175B0F95010090EA174B0F9F7
:106530005010090CE174B0F85010090A217590F858
:106540005000607504E0E42902D00020BDE8F0812D
:106550000120FBE7983B00201C3C0020183900205C
:10656000623200202DE9F0411B4E04460025B6F9A9
:106570000000FAF722F8194F3946F9F7D3FE2074D4
:10658000010A6174010CA174000EE074B6F92800D0
:10659000FAF713F83946F9F7C5FE2075010A617557
:1065A000010CA175000EE075B6F95000FAF705F878
:1065B0003946F9F7B7FE2076010A6176010CA1761B
:1065C000000EE076A52061196D1CEDB20877E42D70
:1065D000F9D30120BDE8F081983B00200000B43BD6
:1065E00072B6012080F31388BFF34F8F054801680E
:1065F000054A01F4E06111430160BFF34F8F00BF12
:10660000FDE700000CED00E00400FA052DE9FF5F56
:1066100083465D4800905D4803904FF0000A5C4857
:106620000290AA228BF800208BF801A0A1238BF8FE
:10663000023011238BF80330D146D04650465546E0
:106640008BF804A069060BEB116400236371A3713E
:10665000009901EB45062DE000EB0801C1EBC101FB
:1066600001EB8102039901EB4201B1F880201AB1DC
:10667000627942F0100205E0B1F87A201AB162792D
:1066800042F001026271009A52896AB1B1F8842025
:106690001AB1617941F0200105E0B1F87C1019B11F
:1066A000617941F002016171401C08F10101C0B241
:1066B00001F0FF08B18E8142CED8002025E000EB2A
:1066C000090101EB011101EB4102029901EB4201C9
:1066D000B1F8C4203AB1617941F080016171A179CA
:1066E00041F055010AE0B1F8BE201AB1627942F0DA
:1066F00008026271B1F8C01009B10121A171401CFA
:1067000009F10101C0B201F0FF09B18A8142D6D876
:10671000002718E007EB0A00401C0190C0B2FBF70D
:106720007DFC012828D00198C0B2FBF777FC002837
:10673000607925D000F0400060717F1C0AF10100F3
:10674000FFB200F0FF0AB08CB842E3D86D1C002005
:10675000EDB2082DFFF476AF0E480068B0F5005F8B
:1067600008D2002001460BEB0002401CC0B2517160
:106770001028F8D3BDE8FF9F607940F00400DBE704
:1067800020F00400D8E7000020310020C02C0020B9
:10679000B6320020180300202DE9F04186B00546EE
:1067A000194F1A4E1A4C14216846F9F758FDB4F8DF
:1067B0001D00DFF8608040BAADF80000207D06289B
:1067C00004D1012241466846FAF764FE012241469F
:1067D0006846FAF751FEBDF80000A7F84000A6F899
:1067E0006000010A2974BDF80000C0B26874627FBD
:1067F000914206D1A17F884203D1012006B0BDE8B5
:10680000F0810020FAE70000C02C0020B632002002
:106810006232002060F00708012002F009FDFBE76A
:106820000EB5F9480190FD490025F848DFF8E493DA
:1068300000900D812F46F64CF74EB9F8002001E08C
:10684000401C088108898242FAD80020DFF8D0B3C2
:1068500008814FF4805A8846322002F0E9FC4FF458
:106860008061F048FCF765F998F8000068B10023F2
:10687000A8F808304146B9F8002001E0401C088122
:1068800008898242FAD888F800300098408830B1F0
:10689000032F7DD0062F7CD0092F7BD04BE1E5BBA9
:1068A000B9F81000D0B30621DF48FDF77BFADE49C6
:1068B000020A8A71C871002251465846FCF741F914
:1068C000502002F093F964230822D749D748FDF7F6
:1068D000F9F8502002F08AF9012251465846FCF797
:1068E00030F9D148007800EB001000EB400004EBD9
:1068F0004000A0F58050B0F8041A052912D9CA4A00
:106900003C21A0F8041A107800EB001000EB4000C6
:1069100004EB4000A0F5805001E012E010E0A0F888
:10692000FC1902E0491CA0F8041ABF490878A0F13C
:106930001102012A01DA401C00E01120087000E079
:106940000325B9F86C0008B1032D06D0062D37D009
:10695000092D4CD00C2D7CD0EFE0B3480621183027
:10696000FDF720FAB049020A18318A71C871002275
:1069700051465846FCF7E5F8502002F037F9AA498D
:10698000642308221831A948FDF79CF8502002E042
:1069900092E09DE0B3E002F029F901225146584609
:1069A000FCF7CFF8B6F87E003C2805D93C20A6F8C5
:1069B0007E00A6F87800C0E0401CA6F87E00BCE08F
:1069C000994806212030FDF7EDF99749020A203158
:1069D0008A71C871002251465846FCF7B2F850201F
:1069E00002F004F9904964230822203158E0B9F8F4
:1069F000120078B30E218E48FDF7D4F98C49020AB3
:106A00008A73C873002251465846FCF79AF8502002
:106A100002F0ECF86423102285498448FDF752F80F
:106A2000502002F0E3F8012251465846FCF789F85D
:106A30007F48007800EBC00101EB4011019800EBAA
:106A40004101A1F58051B1F81006322805D8401C4B
:106A500001E00FE00CE0A1F8100675490878A0F1FC
:106A60002102032A01DA401C00E02120087064E0C2
:106A7000142562E06C4806211030FDF793F96A494D
:106A8000020A10318A71C871002251465846FCF73B
:106A900058F8502002F0AAF8634964230822103104
:106AA0006248FDF70FF8502002F0A0F8012251468D
:106AB0005846FCF746F840E0002251465846FCF79D
:106AC00040F8502002F092F86423082259490AE065
:106AD000002251465846FCF734F8502002F086F860
:106AE0006423554910225148FCF7ECFF502002F076
:106AF0007DF8012251465846FCF723F81BE000229E
:106B0000574651465846FCF71CF8502002F06EF8E4
:106B10004A486423484902884448FCF7D3FF502080
:106B200002F064F8012239465846FCF70AF8009949
:106B30000020074648807F1CFFB2414800680128BA
:106B400020D0B4F8C200401C80B2A4F8C2003C2897
:106B500005D93D20A4F8C2000120A4F8C400B4F86F
:106B60002801401C80B2A4F828013C2805D93D200A
:106B7000A4F828010120A4F82A01032D43D26D1C9A
:106B8000EDB269E62F4A1078112810D0B4F8C2008F
:106B9000401C80B2A4F8C200232805D92420A4F800
:106BA000C2000120A4F8C400107812280DD0B4F857
:106BB0002801401C80B2A4F82801232805D92420EC
:106BC000A4F828010120A4F82A011078A0F11001EE
:106BD0000F2973D85179937900EB001000EB400036
:106BE00043EA012304EB4000A0F580500121029309
:106BF000A0F8041A5078032826D0062824D00120B3
:106C0000A8F80C00DCE0E4E01C4400206232002024
:106C1000B632002020310020983B002000000020E8
:106C2000000C01400010014014010020AC250020A0
:106C3000E0020020D63100201C3200208009002014
:106C40000403002000230020634880780228D6D166
:106C500005216148FDF7A6F802998842CFD1B8F81E
:106C60000C0060BB5C4A0021107800EB001000EBC8
:106C7000400004EB4000A0F58050A0F8FC1910780B
:106C800000EB001000EB400004EB4000A0F580504A
:106C9000A0F8FE195078032811D1D07813460128A6
:106CA0000ED9B8F8080000EB001000EB400004EB30
:106CB000400030F85C2F521C02802AE035E070E082
:106CC000B8F80800142824D200EB001202EB4202AC
:106CD00004EB4202401CA2F85C101A7893F803C03F
:106CE00002EB021202EB420204EB4202A2F58052D6
:106CF000A2F8A0C91A7893F804C002EB021202EBC2
:106D0000420204EB4202A2F58052A2F8C8C9A8F8D8
:106D10000800B8F80820142A01D1A8F8081018783B
:106D2000103880B201F036FD4AE0A0F170010F2961
:106D300038D80123A6F87E305078032804D00628DE
:106D400002D0A8F80C303BE091780829F9D222480B
:106D5000C91CFDF727F8B8F80C00424608BB1E4BCB
:106D6000587803282CD15089142814D20021A6F871
:106D7000781033F8031F49BA26F81010598891FA91
:106D800091FC06EB4001401CA1F828C09B885BBA2F
:106D9000A1F85030508180B2142811D10020A8F8F9
:106DA0000A000DE0A0F120010F2902D8FBF788F9B5
:106DB00006E0E4280AD081380E2801D8FBF7F2F863
:106DC00006490020A8F80C000860D6E6FBF734F965
:106DD000F6E7002540E50000002300200403002022
:106DE0001FB5FB484FF0000B0390DFF8FCC3F948D8
:106DF000FA4E0290ACF80EB0DA465D46F64CF84F0B
:106E0000DFF8E09333880DE006EB4001401C8A8EEA
:106E1000ACF80E0002EB0B011FFA81FB0AF1010135
:106E20001FFA81FABCF80E008342EDD8EE4900202B
:106E3000C881322002F0FCF94FF48061EB48FBF787
:106E400078FEE9480078E0B1DFF89CC34FF0000B12
:106E5000D846ACF80EB033880DE006EB4001401C7C
:106E60008A8EACF80E0002EB0B011FFA81FB0AF1CF
:106E700001011FFA81FABCF80E008342EDD88CF8AC
:106E800000800298DFF86083008830B198F8020033
:106E900003286ED006286DD02EE298F80100002855
:106EA0006BD1B08900286DD00621D148FCF77AFF5C
:106EB000CF49A8F81400020A8A71C87100224FF461
:106EC0000051CC48FBF73DFE502001F08FFE308989
:106ED00001280BD164230822C549C748FCF7F2FDFD
:106EE0003089012802D1502001F080FE0122510397
:106EF000C048FBF726FEBE4A1078C0EBC00000EB8E
:106F0000800004EB4000A0F58050B0F824133C2929
:106F10000ED93C21A0F824131078C0EBC00000EB80
:106F2000800004EB4000A0F58050A0F8181302E0A8
:106F3000491CA0F8241330890028107805D0A0F14E
:106F40003001022917DA401C16E0302801D0302029
:106F500012E098F8030000F13001C9B21170401C32
:106F6000303988F80300022907DB012088F8030084
:106F700003E09AE1BBE13120107098F8010003288A
:106F800003D069E0032188F8011070894FF00601F1
:106F9000012802D088F8011062E09848FCF702FF4F
:106FA0009649A8F81400020A8A71C87100224FF4A9
:106FB00000519048FBF7C5FD502001F017FE3089C5
:106FC000012806D188490A230222491D8A48FCF774
:106FD00079FD6423082289498748FCF773FD3089CD
:106FE000012806D180490A230222491D8248FCF764
:106FF00069FD502001F0FAFD012251037D48FBF7A5
:10700000A0FD7E4A1078C0EBC00000EB800004EBCE
:107010004000A0F50050B0F8C41E3C290ED93C2118
:10702000A0F8C41E1078C0EBC00000EB800004EB99
:107030004000A0F50050A0F8BC1E02E0491CA0F8DA
:10704000C41E1078ABF10101A0F141038B4201DABB
:10705000401C00E04120107098F80100062857D12C
:10706000B6F8640018B1012805D0022855D00920CF
:1070700088F80100C4E05E4806212830FCF792FE43
:107080005B49A8F814002831020A8A71C8710022ED
:107090004FF400515748FBF754FD502001F0A6FD76
:1070A00053496423082228315348FCF70BFD502034
:1070B00001F09CFD012251034E48FBF742FD4C4874
:1070C0002830007800EB800007EBC000A0F580506E
:1070D000B0F8A2133C290ED9454A3C212832A0F829
:1070E000A213107800EB800007EBC000A0F58050E1
:1070F000A0F89C1302E0491CA0F8A2133C492831D7
:107100000878A0F151035DE0401C00E051200870B8
:1071100098F80100092873D0F3E0354806212030A3
:10712000FCF740FE3249A8F814002031020A8A71A7
:10713000C87100224FF400512E48FBF702FD502089
:1071400001F054FD2A496423082220312A48FCF723
:10715000B9FC502001F04AFD012251032548FBF7FC
:10716000F0FC234A1078C0EBC00101EB810104EB75
:107170004101A1F50051B1F8641A3C2912D900EB84
:10718000800007EBC000A0F580503C21A0F8A213BE
:10719000107800EB800007EBC000A0F58050A0F84D
:1071A0009C130AE000EB800007EBC000A0F58050C4
:1071B000B0F8A213491CA0F8A2130D492031087899
:1071C000A0F15003AAF1010293429FDA9CE717E075
:1071D0004028002062320020C02C002020310020F6
:1071E000183900201C3C0020000000200010014045
:1071F0001C010020000C01402C250020F002002082
:10720000B6F86600E8B302F0BDFE0621FD48FCF7C3
:10721000C9FDA8F81400DFF8EC83020A4FF400510E
:1072200088F8062088F807000022F748FBF789FC59
:10723000502001F0DBFC642308224146F348FCF7B0
:1072400041FC502001F0D2FC01225103EE48FBF733
:1072500078FC02F0B7FE98F8001009EBC110A0F519
:107260004050B0F87E103C290CD93C22A0F87E207A
:1072700098F8001009EBC110A0F54050A0F8782054
:1072800003E00EE0491CA0F87E1098F80000A0F181
:107290006002062A01DA401C00E0612088F8000044
:1072A0002FE00C2188F801102BE000224FF4005150
:1072B000D548FBF746FC502001F098FCD4480178F3
:1072C0000D2902D140780A280ED064230822D04923
:1072D000CE48FCF7F7FB502001F088FC0122510357
:1072E000C948FBF72EFC07E064230C22EFE7029A63
:1072F0000020108088F8020098F80210491C88F8D5
:107300000210C4480068012821D0B4F87E00401C57
:1073100080B2A4F87E003C2805D93D20A4F87E0068
:107320000120A4F88000B4F8C400401C80B2A4F886
:10733000C4003C2805D93D20A4F8C4000120A4F8CD
:10734000C600B549487803287ED2401C0DE3B34AF5
:10735000DFF8C48290781044C178007940EA0120B7
:10736000A8F814001078312810D0B4F87E00401C22
:1073700080B2A4F87E00142805D91520A4F87E0058
:107380000120A4F88000107832280DD0B4F8C40091
:10739000401C80B2A4F8C400142805D91520A4F814
:1073A000C4000120A4F8C600505DA0F130010F29EF
:1073B0007DD8C0EBC00000EB800004EB4000974A92
:1073C000A0F580500021A0F81813505DC0EBC0005C
:1073D00000EB800004EB4000A0F58050A0F81A13E9
:1073E000505D0121C0EBC00000EB800004EB4000C9
:1073F000A0F58050A0F8241350190090407803287D
:1074000001D006280BD100988078042807D10721E5
:107410008248FCF7C7FCB8F81420904202D0012043
:1074200088F8040007217D48FCF7BCFCA6F86A0038
:107430000098B0F8030001900098407803286FD1BD
:1074400098F80400002800E08EE2F8D1734800218B
:10745000405DC0EBC00000EB800004EB4000A0F5F5
:107460008050A0F818136D480121405DC0EBC000AA
:1074700000EB800004EB4000A0F58050A0F824133E
:107480006648415D0198F9F733FA64480399405D15
:1074900000EBC00201EBC201A1F5805146F6781263
:1074A000B1F9861291420ED3C0EBC00000E083E038
:1074B00000EB800004EB4000A0F58050B0F81813FA
:1074C000491CA0F81813308920B954480021405DA8
:1074D000F9F78EFAB8F810004246082812D24F4940
:1074E000495D302912D0C1EBC10101EB810104EBF0
:1074F000410101EB4001A1F58051019BA1F8E0326F
:10750000401C108280B208280BD00DE004F55262B6
:1075100002EB4000A0F580500199A0F8001303E0B1
:10752000D7E00020A8F810003C4B0399585D00EB11
:10753000C00201EBC201A1F58051B4F84220B1F9BB
:107540008612C1F1000C944501DC91421CDDC0EBB8
:10755000C00000EB800004EB4000A0F58050B0F8C4
:107560001013491C0904090CA0F81013585DC0EB56
:10757000C00000EB800004EB4000A0F580500ED06E
:107580000121A0F810130BE0C0EBC00000EB80005D
:1075900004EB4000A0F580500021A0F8101300215A
:1075A000585DC0EBC00000EB800004EB4000A0F58C
:1075B0008050A0F81413D1E1A0F140010F297DD82B
:1075C000C0EBC00000EB800004EB4000A0F5805051
:1075D0000021A0F81C13505D0121C0EBC00000EB9E
:1075E000800004EB4000A0F50050A0F8C41E501924
:1075F00000904078032813D0062811D0012088F885
:107600000400ABE14C010020000C01402C250020BF
:1076100090310020FC02002000000020002000200B
:1076200000988078042803D0012188F804100AE02B
:107630000721CF48FCF7B6FBB8F81420904202D0DF
:10764000012088F80400009840780328B3D198F806
:1076500004000028AFD1C648415D0098B0F803008F
:1076600040BAF9F745F9B8F81200434608282AD27B
:10767000DFF8FCC200991CF805200979C2EBC202B0
:1076800002EB820204EB420202EB4002A2F500523E
:107690000902A2F8901E1CF80520DDF800C0C2EB1C
:1076A000C20202EB820204EB42029CF803C002EB2E
:1076B000400241EA0C01A2F5005200E00AE0A2F803
:1076C000901E401C588280B2082802D10020A8F8E1
:1076D000120043E11078A0F150010F297ED8B6F8CE
:1076E0006410012902D0022979D037E100EB800033
:1076F00007EBC0009E49A0F580500123A0F8A233FB
:107700000878002200EB800007EBC000A0F5805055
:10771000A0F89C234878042803D1084680782028C4
:1077200003D0012188F804100AE023219048FCF7D7
:1077300039FBB8F81420904202D0012088F80400E8
:107740008B4841194978042961D198F8041000291F
:107750005DD1884942790A7082794A70C2788A700C
:107760000279CA70425D0B6802EB820207EBC2022B
:10777000A2F58052C2F88033427B0A70827B4A7045
:10778000C27A8A70027BCA70425D0B6802EB820289
:1077900007EBC202A2F58052C2F88833427C0A701D
:1077A000827C4A70C27B8A70027CCA70425D0B6820
:1077B00002EB820207EBC202A2F58052C2F88833C4
:1077C000427D0A70827D4A70C27C8A70027DCA70D6
:1077D000425D02EB820207EBC20201E060E017E0CB
:1077E000A2F580520B68C2F89033427E0A70827E06
:1077F0004A70C27D8A70027ECA70405D096800EBE3
:10780000800007EBC000A0F58050C0F89413A5E0FD
:1078100000EB800007EBC000554AA0F58050012125
:10782000A0F8A2131078002100EB800007EBC00045
:10783000A0F58050A0F89C13507804280BD1104676
:107840008078042807D107211046FCF7ABFAB8F876
:107850001420904202D0012088F8040007214448F7
:10786000FCF7A0FAA6F868004148411949780429B4
:1078700074D198F80410E9BB3E4902790A70C278C5
:107880004A7082798A704279CA70405D096800EB5B
:10789000800007EBC000A0F58050C0F880135DE0C9
:1078A00060380F285AD83448012190F800C009EBFD
:1078B000CC13A3F54053A3F87E100378002109EB05
:1078C000C310A0F54050A0F878105078032802D0DB
:1078D00006287FF493AE264880780228F9D1052146
:1078E0002348FCF75FFAB8F814209042F1D1204801
:1078F000421900E032E05278032A2FD198F80410A0
:1079000061BB415D6139062928D2DFE801F0030936
:107910000F151B21B0F8030041BA09F182001CE0E9
:10792000B0F8030041BA09F1AA0016E0B0F803006C
:1079300041BA09F1D20010E0B0F8030041BA09F5EC
:1079400081700AE0B0F8030041BA09F5957004E0CF
:10795000B0F8030041BA09F5A97001800749002079
:10796000086088F80400ECE400204870FFF761BA72
:10797000002000201C0000204C010020FC02002000
:107980001FB54FF0000BFB4CFB4DDFF8F0A3DFF809
:10799000F093CDF808B0CDF800B00126CDF804B0D2
:1079A000322001F045FC4FF48061F648FBF7C1F846
:1079B000F54800680128F3D1002003909AF80000F0
:1079C0003A2823D19AF80110504633291ED18178E4
:1079D00039291BD1C178302918D100270AEB470873
:1079E00008F10100FCF7B4FAE2498439394408751A
:1079F00008F10100FCF7ACFAE449C8557F1C402FA0
:107A0000ECDB4022DD48F8F711FC00BF00BF524616
:107A10009AF80000392808D05078012805D89078C5
:107A2000952802D8D078502802D95079012803D05F
:107A3000E888401CE8801CE2D079032801D00628A1
:107A4000F6D1D34F0023EB80FB82F88A05EB000CC4
:107A5000115C401C80B28CF80D10F8824028F4D3E1
:107A600098461846FB8280B2115C2154401C80B2BB
:107A7000F8821028F7D303980028DCD1107A4FF64B
:107A8000FF7202EA002068819AF8091008436881B1
:107A9000732877D031DC292864D011DCA0F11000E4
:107AA00018285FD2DFE800F06B5E5E6F5E5E5E5EA0
:107AB0005E5E5E5E5E5E5E5E735E5E5E5E5E5E77B8
:107AC00052287DD00ADC4328E6D002DC402849D188
:107AD00066E0502879D05128F9D18AE07028DBD0AF
:107AE00006DC5328D8D05428D6D05528EFD19BE0B7
:107AF000712867D07228EAD19EE0B0F5BF7F75D0BB
:107B000015DC7A2873D008DCA0F174000628C8D2EE
:107B1000DFE800F09A9FA3A7ABAF7E2868D021DCF6
:107B20007B287BD07C287AD07D281BD1B1E041F224
:107B30009612811A904273D01ADC41F29312A0EB94
:107B4000020190426DD00EDCB0F5C07F6AD0B0F576
:107B5000C87F68D06FF48951C84203D12046FCF732
:107B6000B3FF0290D0E0012972D0022909D1AFE021
:107B7000062906D2DFE801F0C8B4B8BCC0C4FEF7DD
:107B80002FFDC1E05CE08348FEF740FDBCE02046ED
:107B9000FEF77AFA02E02046FCF7D0FC8346B3E019
:107BA0002046F9F715F883464046A7F81680514657
:107BB00080B20A5C2254401C80B2F882402802E065
:107BC0001BE002E034E0F3D39EE0204600F036FDF7
:107BD00083464046A7F81680514680B20A5C22547C
:107BE000401C80B2F8824028F7D38DE059E044E091
:107BF00053E0204600F044FDD0E72046FCF76CFC43
:107C000083464046A7F81680514680B20A5C22544B
:107C1000401C80B2F8824028F7D375E031E034E0B0
:107C20005AE04CE041E044E02046FEF7CDFBB5E7EA
:107C30002046F9F773F8B1E72046FCF7AFFBADE754
:107C40002046FEF7A9FDA9E72046F9F78DF833E0B5
:107C500039E02046FCF7DCFB2EE0204600F036FD44
:107C60002AE02046FBF7B2FF26E02046FCF72EF97B
:107C700022E02046F8F76AFF1EE0204600F076FA80
:107C80008CE72046FCF706F817E02046FCF75AF888
:107C900013E02046FCF72AF80FE02046FBF76CFFC4
:107CA0000BE0204600F036FA07E02046F9F730FCFA
:107CB00002E02046FCF796F883463E7024E020461A
:107CC000FCF72EFD02E02046FDF78EF800901BE049
:107CD0002046FDF74DFAF9E72046FDF78BFBF5E767
:107CE0002046FDF7C9FCF1E72046FDF707FEEDE76A
:107CF0002046FDF745FFE9E72046FEF783F8E5E774
:107D00002046FEF72FFC0190688913281AD00098AE
:107D100070B30020009094212046FCF743F8010A3C
:107D200084F8941084F89500002210214F464846AC
:107D3000FAF707FF502000F059FF02F023F99623CD
:107D40001A4643E03E211348FCF72CF81149020A79
:107D50004F4601F83E2F0022487010214846FAF79E
:107D6000F0FE502000F042FF64234022094973E0F6
:107D700012E00000E001002062320020002200201A
:107D80000008014000100140000300206C26002084
:107D900000000020002400200198F0B10020019094
:107DA00060212046FBF7FEFF010A84F8601084F88A
:107DB0006100002210214F464846FAF7C2FE5020CB
:107DC00000F014FF02F0DEF89623622221462B48D1
:107DD000FBF778FE02F0F6F841E00298E8B10020E7
:107DE000029084F8E88084F8E980EA212046FBF7D5
:107DF000D9FF010A84F8EA1084F8EB000022102170
:107E00004F464846FAF79DFE502000F0EFFE02F084
:107E1000B9F84FF4FA73EC22D8E7BBF1000F01D0A8
:107E2000404600E0FF2084F83C0084F83D003E21FD
:107E30002046FBF7B7FF010A84F83E1084F83F00A4
:107E4000002210214F464846FAF77BFE502000F0F2
:107E5000CDFE6423402221460848FBF733FE502024
:107E600000F0C4FE012210213846FAF76AFE4FF0F6
:107E7000000B03490020086092E500006C250020FB
:107E800000030020184D194FDFF864904FF480680C
:107E900041464846FAF74DFEF8F7FEFD00241FE084
:107EA000052C04D2DFE804F0030507090900114995
:107EB00004E0114902E0114900E0114904EB840695
:107EC000224655F83600F8F78FFF05EBC6018861AA
:107ED0002046F9F7C1F9642001F0AAF9641CE4B264
:107EE0003888A042D4D9DBE718390020203100209F
:107EF0000010014040030020D00400206006002054
:107F0000F0070020012001F093F9FBE7012001F0C8
:107F10008FF9FBE7012001F08BF9FBE7012001F06D
:107F200087F9FBE7012001F083F9FBE7012001F06D
:107F30007FF9FBE70B4E0A4CDFF82C804FF4FA7503
:107F40003715284601F074F9A0690121401CA06191
:107F50003046FAF7EEFD39464046FAF7EAFDF0E71B
:107F600000000020000801400010014010B5502022
:107F700080F31188BFF34F8FBFF36F8F02F0AAFD1C
:107F800018B104494FF080500860002080F3118838
:107F900010BD000004ED00E030B58FB02821684628
:107FA000F8F75DF914210AA8F8F759F9012001043E
:107FB00000248DE8130004904FF4E010CDE9081080
:107FC000022507956846FAF791FF08B172B6FEE7F9
:107FD0000F20CDE90A054FF48060CDE90C40022165
:107FE0000AA80E94FAF770FE002801D072B6FEE7D8
:107FF0000FB030BD704700000148FBF733BA0000F6
:108000005C2400200148FBF72DBA0000A4240020C6
:108010000148FBF727BA0000B8270020F0B5026836
:108020001C4D1D4E1D4FDFF878C01E4B4FF0804E8B
:10803000A84209D0984207D0704505D0B04203D07D
:10804000B84201D0604503D122F070044A6822434F
:10805000A84209D0984207D0704505D0B04203D05D
:10806000B84201D0604503D122F44074CA6822436B
:108070004C6922F08002224302608A68C2620A6868
:108080008262A84201D0984201D1096901630121AD
:108090004161F0BD002C0140000400400008004098
:1080A000000C00400034014010B5846842EA03220D
:1080B00024F47F440A432243826010BD826822F088
:1080C00070020A4342F007018160704710B5046AEC
:1080D000036A23F001030362836923F0F00343EA98
:1080E000021324F00A020A438361026210BD10B534
:1080F000036A23F0100303628469036A24F4704462
:1081000044EA023223F0A00343EA011182610162D2
:1081100010BD0000124B30B4997C4FF6FF7404EA96
:108120000122D97C0D481143032914D1418800292B
:1081300011D1017D06290ED101214180187D5A7D82
:10814000084904EA002002430A8030BC03F116010A
:108150000548F8F76BB830BC704700006232002069
:1081600000220020800900201C320020F0B58BB0D6
:1081700005461C4E1C4C28216846F8F770F8B4F8E8
:108180001D001A4F40BAADF80000207D062804D12A
:10819000012239466846F9F77DF9012239466846D9
:1081A000F9F76AF9BDF80000000A2874BDF800006C
:1081B0006874BDF80000A0F57F41FF3901D0A6F832
:1081C0006600287C617F884206D1687CA17F884256
:1081D00002D1207D062802D000200BB0F0BD012086
:1081E000FBE70000203100206232002048F0070841
:1081F00010B501F045FE002805D0D0E90012BDE819
:1082000010401046084710BD10B5406A0021C185D6
:10821000C184FBF714FA10BD70B5446A2068406948
:1082200094F83910C0F3C0100025212904D118B1E9
:10823000E584204600F046F82068406994F83A103A
:10824000C0F38010222904D118B1E585204600F042
:108250002BF8E06B40F01000E0632046FBF7EFF9ED
:1082600070BD10B50146406A09680968890613D4D3
:108270000021C1850168CA6822F48072CA60016861
:108280004A6922F001024A6101684A6922F040020B
:108290004A61202180F83A10FBF712FC10BD10B59E
:1082A000406AFBF70EFC10BD0168CA6822F49072A8
:1082B000CA6001684A6922F001024A61202180F8FF
:1082C0003A1070470168CA6822F0C002CA602021D3
:1082D00080F83910704710B590F83A10222901D073
:1082E000022010BD81684FF48053994201D1026988
:1082F00022B1826A99421BD049B10AE00268816AC0
:108300005268C2F308020A80816A891C08E0016988
:1083100071B10168496801F07F011170816A491CDF
:108320008162C18D491E0904090CC18503D016E084
:1083300001684968F1E70168CA6822F02002CA6052
:108340000168CA6822F48072CA6001684A6922F032
:1083500001024A61202180F83A10FBF7B1FB0020AE
:1083600010BD000070B5044600680169E26821F4A0
:10837000405111430161A1682069014360690143D3
:108380002068C26841F20C639A430A43C2602068C5
:108390004169A26921F44071114341611E4920687D
:1083A000884202D1FAF75CFD01E0FAF749FD00EBE3
:1083B000C00101EB0011606864228000B1FBF0F3A2
:1083C000B3FBF2F36FF018067343B1FBF0F5B1FBAA
:1083D000F0F605EB8305322303EB0515B5FBF2F54B
:1083E000B6FBF2F605F0F00505EB0615B1FBF0F66D
:1083F000B1FBF0F0B0FBF2F06FF01801484306EB70
:10840000800003EB0010B0FBF2F0216800F00F00D9
:108410002844886070BD0000003801402DE9F0411B
:108420001E46174688460446069D1CE0681C1AD066
:1084300025B1FAF78BFB801BA84214D92068C168CC
:1084400021F4D071C1602068416921F001014161CE
:10845000202084F8390084F83A00002084F838009D
:108460000320BDE8F0812068016838EA010004D0EB
:108470000020B842DAD00020F3E70120F9E700003D
:1084800038B51448FBF7DCF8124800680168C943A6
:10849000C9061DD40168406800900E48FBF7A3F898
:1084A0000D48006840680D4CC0F580720C490D48BD
:1084B0006261F7F7BBFE4FF4807529460848F7F76D
:1084C000CEFE2A4606490348FBF7AEFA012020609B
:1084D00038BD00002C250020940F0020FC02002055
:1084E000100D00200020002038B51448FBF7A8F834
:1084F000124800680168C943C9061DD40168406874
:1085000000900E48FBF76FF80D48006840680D4C6E
:10851000C0F580720C490D48E260F7F787FE4FF412
:10852000807529460848F7F79AFE2A460649034807
:10853000FBF77AFA0120606038BD00006C2500204E
:1085400030270020FC020020002100200022002013
:1085500038B51448FBF774F8124800680168C9433D
:10856000C9061DD40168406800900E48FBF73BF82F
:108570000D48006840680D4CC0F580720C490D48EC
:108580002261F7F753FE4FF4807529460848F7F744
:1085900066FE2A4606490348FBF746FA0120A0601A
:1085A00038BD0000AC25002074270020FC0200200C
:1085B000100E002000230020FEE7000070B58AB0F6
:1085C0001A4D28216846F7F74AFE0024012218496F
:1085D0006846F8F751FFBDF800004FF6FF76B0424D
:1085E00000D0A880082213496846F8F745FF69467D
:1085F00008E031F81400B04202D005EB440290824A
:10860000641CE4B22888A042F3D800200A4907E09D
:1086100005EB40020B88928A401C1A440A80C0B2C3
:108620002A888242F4D80AB070BD000020310020B0
:1086300028F0070800E00708200300200F4810B5C5
:10864000418811B9017D062901D0002010BD0B4CD5
:10865000012141808C3C807F2070062060700020CA
:108660000222A070E2702071617120460621FBF7A2
:1086700099FB010AA171E071012010BD6232002056
:10868000114910B54A8812B90A7D062A01D0002086
:1086900010BD0D4C01224A808C3C887F2070062042
:1086A00060700020A0701020E070C87F207191F8E9
:1086B0002000607120460621FBF774FB010AA171BE
:1086C000E071012010BD0000623200202DE9F04170
:1086D0008AB006462B4D2C4C28216846F7F7BFFD83
:1086E00000206F4605E02118497F27F81010401C34
:1086F000C0B2217E8142F6D8207DDFF89080062826
:1087000004D1012241463846F8F7C4FE0122414611
:108710006846F8F7B1FEBDF800003074BDF80000FF
:10872000052800D2A880207DDFF86480062804D1C7
:1087300008224146B81CF8F7ADFE08224146B81C95
:10874000F8F79AFE002013E007EB40022318518847
:108750009B7F994202D0237D062B10D0082905D299
:1087600005EB40039982917832185174401CC0B2D5
:10877000217E8142E8D801200AB0BDE8F0810020C6
:10878000FAE70000203100206232002028F00708BC
:1087900000E00708C0B210B5264900EB001000EB5E
:1087A0004000244C31F810300122002104EB40003D
:1087B000012B01D07BB11CE0A0F85210B0F8503072
:1087C0005B1C9BB2A0F85030022B12D3A0F85010C3
:1087D000A0F858200DE0A0F85010B0F852305B1C03
:1087E0009BB2A0F85230022B03D3A0F85210A0F88D
:1087F0005810038D012B0FD0002B0CD1A0F8541072
:10880000B0F85620521C92B2A0F85620022A02D389
:1088100020F8561F818010BDA0F85610B0F85430D3
:108820005B1C9BB2A0F85430022BF4D320F8541FE9
:10883000C28010BDB63200200FB4084B10B504A999
:1088400002AA039800F02CF8044602A9002000F0C8
:10885000C8F9204610BC5DF814FB0000E38B00084B
:108860000907090E002804DB00F1E02080F800145D
:10887000704700F00F0000F1E02080F8141D7047F1
:1088800002E008C8121F08C1002AFAD170477047D9
:10889000002001E001C1121F002AFBD17047000037
:1088A0002DE9FF4F8BB088460546002606E02528B7
:1088B0000BD0DDE90D1290476D1C761C287800283E
:1088C000F5D10FB03046BDE8F08F0024A146A24696
:1088D0000122AE4900E0044315F8013F203B02FAB3
:1088E00003F00842F7D128782A2810D06FF02F0221
:1088F0002878A0F13001092915D809EB890102EB8C
:10890000410144F0020400EB01096D1CF0E758F846
:10891000041B5FEA010903D544F40054C9F10009BE
:1089200044F002046D1C28782E2817D115F8010F89
:1089300044F004042A280ED06FF02F022878A0F10A
:10894000300109290AD80AEB8A0102EB410100EB48
:10895000010A6D1CF2E758F804AB6D1C28786C28EE
:108960000FD006DC4C2817D068280DD06A2814D107
:1089700004E0742810D07A280FD10DE044F40014DC
:108980000AE044F4801401E044F440146978814220
:1089900002D104F580146D1C6D1C2878692865D0FF
:1089A00006DC00288DD0632827D0642806D15DE03E
:1089B0006E2808D073282AD0752877D0DDE90D12EB
:1089C0009047761CE0E0C4F30250022809D0032847
:1089D0000DD0D8F8001004280DD00E6008F104085E
:1089E000D2E0D8F80010F217C1E90062F6E7D8F833
:1089F00000100E80F2E70E70F0E718F8041B8DF8F7
:108A0000001000208DF80100EB46012003E058F82B
:108A100004BB4FF0FF3061074FF0000701D40AE0BC
:108A20007F1C57450DDA8742FADB1BF80710002937
:108A3000F6D106E07F1C8742FCDB1BF807100029FB
:108A4000F8D1DDE90D23A9EB07008146214600F0AE
:108A5000B1F83044C61904E0DDE90D121BF8010B32
:108A600090477F1EF8D22146484688E058F8040B0C
:108A7000C4F302514FF00A0B032900D100B20429BC
:108A800000D140B2002802DA40422D2102E0210547
:108A900005D52B218DF82410012104E006E0E10723
:108AA00010D02021F6E708AF089113E058F8040B26
:108AB000C4F302514FF00A0B032900D180B20429FC
:108AC00000D1C0B20021EEE75946F7F7EBFD303197
:108AD00007F8011D0028F7D1ADEB070000F1200BCE
:108AE000600702D524F4803401E04FF0010ADA4532
:108AF00002DDAAEB0B0000E00020824600EB0B0138
:108B000008980144A9EB01000A90E00306D4DDE9CE
:108B10000D2321460A9800F04DF806444FF0000955
:108B200008E009A911F80900DDE90D12904709F1E3
:108B30000109761C08998945F3DBE0030CD5DDE9D2
:108B40000D2321460A9800F035F8064404E0DDE9DB
:108B50000D1230209047761CBAF10001AAF1010AEB
:108B6000F5DC05E0DDE90D1217F8010B9047761CE6
:108B7000BBF10001ABF1010BF4DC0A982146DDE901
:108B80000D2300F005F806446D1C97E60928010046
:108B90002DE9F041044600251E461746880404D4FA
:108BA00005E039462020B0476D1C641EF9D52846E3
:108BB000BDE8F0812DE9F041044600251E469046AF
:108BC000C80301D5302700E02027880404D505E03C
:108BD00041463846B0476D1C641EF9D52846BDE8AD
:108BE000F0810A68531C0B6010707047C1000020B0
:108BF00001E000BF401C8842FBD370472DE9F041E3
:108C0000C1F30A52A2F2FF362F4A304B0D460446FA
:108C1000142E2FDA002E12DAF7F7B6FB00221346D5
:108C2000F7F70CFE4CD2002DA4BF0024254647DAEE
:108C300025F00040204318BF254D41D018E0DFF853
:108C400094C02CFA06F705EA070C5CEA040C08BF8E
:108C5000BDE8F081F7F798FB00221346F7F7EEFD29
:108C60002ED2002D03DA4FF48010F0400544BD43AE
:108C7000002425E0332EC8BFBDE8F081A6F1140C16
:108C80004FF0FF3727FA0CF73C4208BFBDE8F081F0
:108C9000F7F71EFC00221346F7F7D0FD10D2002D87
:108CA0000DDA142E08BF6D1C09D0C6F13400012165
:108CB00001FA00F02044A04238BF6D1C0446BC43BA
:108CC00029462046BDE8F0819C7500883CE4377E4B
:108CD0000000F0BFFFFF0F0086B000240094019455
:108CE00002940394F9F740FFF8F7FEF8FBF7F4FA63
:108CF000FFF764FCF7F7C8FFFFF74EF9FBF742F9FF
:108D0000FE48416941F001014161416901F0010101
:108D10000491416941F0020141614069002200F083
:108D20000200049005210E20F9F79CFF0E20F9F7B0
:108D30008BFF002205213B20F9F794FF3B20F9F738
:108D400083FFFBF74FFAEF48ED4901604FF4E13143
:108D5000C0E901140C21C460C0E904418461C4610C
:108D6000FAF71CFD08B172B6FEE7FBF763FAFBF7F2
:108D700089FAE649E44808600846F9F717FA08B1A5
:108D800072B6FEE7DF490494A439E148059408600F
:108D90000846F9F758FA08B172B6FEE73C20CDE96B
:108DA0000404D848102204A9A438F9F725FA08B118
:108DB00072B6FEE7FBF7AEF9FBF7E2F9FBF766F9EF
:108DC0000122D44E550329463046F9F7BAFE012256
:108DD000170339463046F9F7B4FEDFF83C83012229
:108DE00010214046F9F7ADFEE81000900120CDE9D2
:108DF0000104022003906946C848F9F79DFD00224E
:108E000029463046F9F79DFE002229463046F9F7FB
:108E100098FE002239463046F9F793FE00221021D1
:108E20004046F9F78EFE0220F9F7C0FC2021BC482D
:108E3000F7F715FA0522BBA1B948FFF7FDFCB849C1
:108E400082B24FF49673A1F18000FAF73BFE012243
:108E500029463046F9F775FE012239463046F9F7C2
:108E600070FE012210214046F9F76BFE00F01CFA5B
:108E7000B14800F08FFAA54CD43C2061AE481030C8
:108E800000F088FA6061AC48203000F083FAA061FD
:108E9000A948303000F07EFAE061A748403000F089
:108EA00079FA2062A448503000F074FA6062A24857
:108EB000603000F06FFAA0629F48703000F06AFAEC
:108EC000E0629D48803000F065FA20639A48903057
:108ED00000F060FA60639848A03000F05BFAA0638D
:108EE0009548B03000F056FA934A0121E063C03251
:108EF000084600F08FFA904A01212064D0320846DB
:108F000000F088FA8C4A01216064E032084600F0E3
:108F100081FA894A0121A064F032084600F07AFA09
:108F20000121E064854A084600F074FA834A012171
:108F300020651032084600F06DFA804A0121606514
:108F40002032084600F066FA7C4A0121A0653032E2
:108F5000084600F05FFA794A0221E065403208468F
:108F600000F058FA754A022120665032084600F097
:108F700051FA724A022160666032084600F04AFAED
:108F80006E4A0221A0667032084600F043FA6A4B2E
:108F9000E066A03B00220121694800F0EDFAA4F14F
:108FA0008005654BA866903B00220121654800F0D2
:108FB000E3FA614BE866803B00220121624800F041
:108FC000DBFA5D4B2867703B002201215F4800F00F
:108FD000D3FA594B6867603B002201215C4800F0DE
:108FE000CBFA554BA867503B00220121594800F0AD
:108FF000C3FA514BE867403B00220121564800F07C
:10900000BBFA4D4B2060303B00220121534800F059
:10901000B3FA494B6060203B00220121504800F028
:10902000ABFA454BA060103B002201214D4800F0F7
:10903000A3FAE0604C4A0221102000F071F94A4A7C
:10904000286518320221102000F06AF9464A686546
:1090500030320221102000F063F9434AA8654832FB
:109060000221102000F05CF93F4AE86560320221DD
:10907000102000F055F93C4A286678320221102071
:1090800000F04EF96866394A0021394800F022FAAA
:10909000364A286224320021364800F01BFA334A4F
:1090A000686248320021344800F014FA2F4AA8625E
:1090B0006C320021314800F00DFA2C4AE8629032FF
:1090C00000212F4800F006FA284A2863B432002114
:1090D0002C4800F0FFF9244A6863D83A00212A4856
:1090E00000F0F8F9204AA863B43A0021274800F0BC
:1090F000F1F91D4AE863903A002149E0001002406E
:1091000000500040EC2400200030024054010020B8
:1091100000740040000C01400008014000100140B4
:10912000EC2500207379737974656D207265736521
:10913000742E2E2E2535640050B3000850B400085C
:10914000D50E0008D90E0008DB0E0008DD0E000861
:10915000DF0E0008E10E0008E30E0008E50E00082F
:10916000E70E0008D70E000820B2000870B0000813
:109170001968000821680008E16D0008817900087D
:10918000857E0008057F00080D7F0008157F000818
:10919000214800F09FF92864204A0021204800F06F
:1091A00099F91E4A6864243200211E4800F092F9A1
:1091B0001A4AA864483200211B4800F08BF9E86481
:1091C0001A4800F04FF820671848103000F04AF8AD
:1091D00060671648203000F045F8A067134830302B
:1091E00000F040F8E0671148403000F03BF8803470
:1091F00020600E48503000F035F860600B48603059
:1092000000F030F8A0600948703000F02BF8E06002
:1092100000F066F8FEE700001D7F0008B4B100080A
:10922000257F00082D7F0008357F0008D0B4000896
:1092300010B5EFF3058149B9EFF3108131B9084951
:109240000968022905D1EFF3118111B16FF005040E
:1092500003E0002408B100F093FF204610BD000099
:10926000E809002010B54FF00001EFF30582BAB90C
:10927000EFF31082A2B90B4A1268022A02D1EFF36F
:1092800011826AB948B1D0E902202AB1202807D357
:10929000104601F067F802E010B901F055F80146F8
:1092A000084610BDE8090020EFF3058058B9EFF338
:1092B000108040B909490868022801D030B109E09E
:1092C000EFF3118030B16FF00500704701200860A6
:1092D000002070474FF0FF3070470000E809002081
:1092E00010B5EFF3058060B9EFF3108048B90B4972
:1092F0000868022802D0012806D00BE0EFF31180A5
:1093000040B16FF0050010BD0220086000F0A0FF22
:10931000002010BD4FF0FF3010BD0000E809002014
:10932000F8B514464FF00005EFF305826ABBEFF382
:10933000108252BB164A1268022A02D1EFF3118240
:109340001ABB10B309B3ACB1D4E902326BB1502AE5
:109350001BD32269CAB1676900FB01F6B74214D377
:109360000025009501F0E1F807E072B9226962B9C1
:10937000626952B9002201F0B4F8050005D00CB1C1
:10938000216800E0002100F09BFE2846F8BD0000A7
:10939000E809002070B505464FF00004EFF30580A2
:1093A000A0BBEFF3108088BB19480068022802D1E7
:1093B000EFF3118050BB0DB1686800E00020C107D9
:1093C00001D0012600E0002600071FD46DB1D5E9C9
:1093D000021021B1502819D31EB1042002E020B19F
:1093E00014E0012001F070F805E00EB1042000E067
:1093F000012001F05EF8040008D00DB1296800E0FA
:10940000002100F05DFE0EB144F00104204670BD65
:10941000E8090020F8B514460E464FF00005EFF3BA
:109420000581E9BBEFF31081D1BB29490968022905
:1094300002D1EFF3118199BB90B3864245D84FF02A
:10944000FF3244B1A1680029E16803D0502903D359
:10945000012201E001B90022511C36D0012809D0B7
:10946000012A29D0314600F0E7FF05002DD044B392
:10947000216827E0012A16D003220021012001F0F3
:1094800030F8050021D0002EF1D000231A461946ED
:1094900001F0C2F80128EAD0284600F023FE00E0DF
:1094A00013E0002511E00320009000221146012066
:1094B000A36801F03AF8E4E73146A26800F0D9FF6A
:1094C000D3E70021284600F0FBFD2846F8BD000048
:1094D000E8090020F0B585B00B464FF00005EFF32A
:1094E00005810395A1BBEFF3108189BB2149096870
:1094F000022902D1EFF3118151BB48B38026182114
:109500008DF8105004AC42B3176807B13C46976918
:1095100007B139464F1E382F02D21779FF0702D004
:10952000002005B0F0BD576907B1BE08D2F808C0E9
:10953000BCF1000F0DD0D5685C2D18D312693AB17B
:1095400037B18DE806103246214601F082FA0390C9
:109550000DE0D7685FB912694AB903AACDE90012D4
:10956000B2B2214601F048FA012800D003950398D1
:10957000D7E70000E80900202DE9FC411C4617460A
:10958000884606464FF00005EFF3058078BBEFF301
:10959000108060BB17480068022802D1EFF31180E9
:1095A00028BB26B3082000F0FFFB03001FD0B8F152
:1095B000000FC3E9006711D001220F4E00208CB1CB
:1095C000216801B10846A16851B1E468302C0ED37E
:1095D000CDE90061012101F0D1FB07E00022ECE7B9
:1095E000E16821B90121009601F0AEFB054628464D
:1095F000BDE8FC81E8090020F18100082DE9F04177
:10960000154E0F46044675693168002081F85A00EE
:109610003068001D00F058FC601C07D137B131687C
:10962000BDE8F0410D48091D00F09FBC30682C4496
:10963000AC424460316805D2B068BDE8F041091D14
:1096400000F07BBC7068091D00F077FC306B844231
:1096500000D23463BDE8F08198090020AC570020A7
:109660002DE9F041054600F08DFC2D4E3069401C7F
:10967000306130682B4F10B1F06930B32BE03560AA
:109680003069012827D1002404EB840007EB800017
:1096900000F045FC641C382CF6D3234800F03FFC56
:1096A0002148143000F03BFC1F48283000F037FC04
:1096B0001D483C3000F033FC1B48503000F02FFCBC
:1096C000194870601430B06005E03068E96AC06A1B
:1096D000884200D83560F06A401CF0626864E86A2D
:1096E000B169884200D9B06100EB800007EB8000CF
:1096F000291D00F03AFC00F065FCF06900280CD050
:109700003068E96AC06A884207D208494FF0805041
:109710000860BFF34F8FBFF36F8FBDE8F08100008B
:1097200098090020FC5200205C57002004ED00E066
:1097300038B500F027FC104CA068C8B90F4800F0FD
:10974000EEFB0E48143000F0EAFB0C4820601430A9
:1097500060600A4B00202833009003F15002102172
:109760000A2000F0E2FEA06010B105A100F0A8FC04
:10977000BDE8384000F026BCD4090020C0570020C6
:10978000546D72510000000030B4026C0B46002A88
:109790000BD0C1681144C1604468A14201D3016883
:1097A000C16030BC1846F6F741BD30BC70472DE9AA
:1097B000F041856B174604460026026C82B1C7B1A2
:1097C000E068F6F733FDE168206C091AE160226871
:1097D000914202D26168081AE060022F16D017E0A9
:1097E0002068A8B9606801F0D9F9064600206060D9
:1097F0000EE0A068F6F71AFD216CA0680844A0608E
:109800006168884204D32068A06001E005B16D1E44
:109810006D1CA5633046BDE8F08110B5044690F894
:10982000590058B101280CD002280FD0502080F3E5
:109830001188BFF34F8FBFF36F8FFEE7206B00F0EF
:10984000D5FB2046BDE8104000F0D0BB10BD0000A5
:1098500010484FF48041420706D0C01D0D4920F04A
:109860000700411AC1F580410B4A00230144C2E9B7
:1098700000030839103A21F0070111604B600B60BA
:109880000B1AC0E9001393604FF000405360D060A2
:1098900070470000905F0020FC090020144E154D19
:1098A000A6F29C474FF08058DFF84C9011E000F092
:1098B00069FBF068C468201D00F006FB2869401EA3
:1098C0002861E868401EE86000F07CFB2046FFF756
:1098D000A4FFE8680028EAD13868012805D9C9F84A
:1098E0000080BFF34F8FBFF36F8F00F017FBF0E7DF
:1098F000985700209809002004ED00E0002807D0C8
:109900000021416001600B460A46C16000F084BE40
:10991000704770B51D46049C49B12260C4E90F012F
:109920000121204600F034FE84F84C5070BD2460C4
:10993000F4E72DE9F0470E46DDE909841746824633
:1099400091009946089DA522206BF6F781FC6FF0E7
:109950000301206B01EB8701084420F0070778071B
:1099600007D0502080F31188BFF34F8FBFF36F8F64
:10997000FEE72218315C82F83410315C11B1401CD2
:109980001028F6D3002684F84360382D00D33725FD
:10999000E562C4E91356201D00F0CCFA04F118006A
:1099A00000F0C8FA2461C5F138006462A061666500
:1099B00084F8586084F85A604A465146384600F0A8
:1099C00071FA2060B8F1000F01D0C8F80040BDE87E
:1099D000F0872DE9F0471E46DDE9089417460D0093
:1099E00080460ED0002C14D0FFF7A2FEC4F80080F1
:1099F000C4E90657C4E90869201DBDE8F04700F036
:109A000099BA502080F31188BFF34F8FBFF36F8F47
:109A1000FEE7BDE8F087000030B5114900E01146CF
:109A20000A688242FBD34B685C18844203D14068C9
:109A300018444860084643681C18944209D1084CF1
:109A4000103C2468A24209D052681A4442600A6855
:109A500012680260814200D0086030BD0460F9E7FE
:109A6000FC09002070B5002441600B4D006191425B
:109A700006D8D11A8269914206D2011D686807E0B2
:109A80009A4203D2994201D3012403E0011D2868C0
:109A900000F053FA204670BDD409002010B50446EA
:109AA00000F070FAA06B20B1002400F08BFA204681
:109AB00010BD0124F9E7000030B587B0304D55E006
:109AC0000198002806DADDE90301029A904701981F
:109AD00000284BDB039C606910B1201D00F0F4F9F5
:109AE00005A800F0B9F8024601980A283ED2DFE83E
:109AF00000F00505053D263705053D260298A169BC
:109B0000034601442046FFF7ADFF00B3616A2046DB
:109B10008847E069012829D1002000900298A169B6
:109B2000002342181946204601F070F978B95020F8
:109B300080F31188BFF34F8FBFF36F8FFEE702985A
:109B4000A06128B1811813462046FFF78BFF0DE076
:109B5000502080F31188BFF34F8FBFF36F8FFEE764
:109B600094F82C0010B9204600F040FA002201A918
:109B7000A86800F061FE0028A2D107B030BD000047
:109B8000D40900202DE9FC410E46054600F0A2FB59
:109B900001A800F061F80446019818B101F074F8CA
:109BA000BDE8FC81224FAEB178680068A8B30026FA
:109BB000291B3246B86800F0C1FA01F065F80028A8
:109BC000EED11C494FF080500860BFF34F8FBFF3B8
:109BD0006F8FE5E7A542EBD801F056F838682646C6
:109BE000C068C468201D00F06FF9E069012810D139
:109BF000A0692B46411932462046FFF733FF40B19A
:109C000000200346014600902A46204601F0FEF857
:109C100020B1616A20468847C2E707E0502080F300
:109C20001188BFF34F8FBFF36F8FFEE70126BFE7A9
:109C3000D409002004ED00E006484168096829B114
:109C40004168C968C9684968016370474FF0FF31CE
:109C5000FAE700009809002070B5054600F034FFCF
:109C6000064E04463069844203D200F009F8012010
:109C700000E0002028602046346170BDD409002037
:109C8000F8B5194E1FE0C068C4680568201D00F0D3
:109C90001BF9616A20468847E069012813D1A06951
:109CA0002844A84206D924616060211D306800F074
:109CB00044F908E000200346014600902A46204669
:109CC00001F0A4F838B1306801680029DBD171686F
:109CD000C6E90010F8BD502080F31188BFF34F8F04
:109CE000BFF36F8FFEE70000D409002008484068EA
:109CF000401C4FF0500080F3118804D0BFF34F8F09
:109D0000BFF36F8FFEE7BFF34F8FBFF36F8FFEE799
:109D1000040A0020084C2068016839B1002139B1DB
:109D20000020FFF72FFFFFF7C7FEF4E70121F6E75A
:109D3000C0680068F5E70000D40900202DE9F04173
:109D4000044600F01FF994F9455004F1240609E097
:109D5000606A48B1304600F05FFF08B100F03EFA9B
:109D60006D1E6DB2002DF3DC4FF0FF3684F84560B8
:109D700000F028F900F006F994F9445004F11007B6
:109D800009E0206948B1384600F046FF08B100F00C
:109D900025FA6D1E6DB2002DF3DC84F84460BDE839
:109DA000F04100F00FB900002DE9F0410546002612
:109DB00000F090FA314F386808B9FFF749FDF868AC
:109DC00005424BD1C5B3083568070ED005F0070032
:109DD000C0F108000544680707D0502080F31188BF
:109DE000BFF34F8FBFF36F8FFEE72DB378688542C7
:109DF00034D8224910310846046801E0214604465F
:109E00006068A84202D220680028F7D138688442EE
:109E100024D00E682068086060680836411B10294D
:109E20000FD96019420708D0502080F31188BFF382
:109E30004F8FBFF36F8FFEE710E041606560FFF763
:109E4000EBFD61687868401A7860BA68904200D289
:109E5000B860F86801430020C4E9000100F014FF75
:109E6000700707D0502080F31188BFF34F8FBFF3E6
:109E70006F8FFEE73046BDE8F0810000EC0900205E
:109E800010B5040006D000F07DF8246A00F09AF8BE
:109E9000204610BD502080F31188BFF34F8FBFF3D1
:109EA0006F8FFEE710B5031F4FF080741C601B1FFF
:109EB00021F001011960191F024B0B601439403861
:109EC0000A6010BDED9C0008D0E9013201699A607A
:109ED000D0E901235A604A68824201D182684A600F
:109EE000002202610868401E086008687047000090
:109EF000034B036003F15C00086080201060704732
:109F0000D8580020044B036003F15C0008604FF454
:109F10008070106070470000345B0020704700F1D3
:109F200008014FF0FF32C0E90112C1600161002158
:109F30000160704700210161704730B50C68621CF8
:109F400002D000F1080202E0026904E01A465368F8
:109F50001D68A542FAD953684B6099608A605160C8
:109F600008610168491C016030BD42684A6093681D
:109F70008B6093685960916008610168491C0160B9
:109F800070470000502080F31188BFF34F8FBFF35C
:109F90006F8F0A494868401C486001280CD1084866
:109FA000006810F0FF0F07D0502080F31188BFF336
:109FB0004F8FBFF36F8FFEE770470000040A002049
:109FC00004ED00E00849486828B1401E486001D10E
:109FD00080F311887047502080F31188BFF34F8FB2
:109FE000BFF36F8FFEE70000040A002070B5002861
:109FF00027D0144DA0F108046068E968084207D131
:10A00000502080F31188BFF34F8FBFF36F8FFEE7AF
:10A0100022683AB1502080F31188BFF34F8FBFF30D
:10A020006F8FFEE78843606000F054F960686968EC
:10A03000084468602046FFF7EFFCBDE8704000F080
:10A0400023BE70BDEC0900204FF0E020002101612B
:10A05000816105494FF47A720968B1FBF2F1491E3A
:10A0600041610721016170478809002010B5F6F7AA
:10A07000B1F8114910280ED300F1E02090F8F00358
:10A080000A78904207D2502080F31188BFF34F8F97
:10A09000BFF36F8FFEE709480068896800F4E0604D
:10A0A000884207D9502080F31188BFF34F8FBFF348
:10A0B0006F8FFEE710BD0000040A00200CED00E0E9
:10A0C00010B5074B002253F832401CB1521C082A2D
:10A0D000F9D310BD43F8321003EBC201486010BD44
:10A0E000BC52002010B504000AD000F013F894F818
:10A0F000460000280CD12046BDE81040FFF776BF8F
:10A10000502080F31188BFF34F8FBFF36F8FFEE7AE
:10A1100010BD0000084A002102EBC1035B688342C6
:10A1200006D1002042F8310002EBC10148607047BF
:10A13000491C0829F0D37047BC52002070B5154661
:10A140000E460446FFF71EFF94F944100020491CF8
:10A1500001D184F8440094F94510491C01D184F8D8
:10A160004500FFF72FFFA06B28B92A46314604F1BE
:10A17000240000F051F82046BDE87040FFF7DEBD36
:10A1800010B5020014D00F48806B38B1502080F316
:10A190001188BFF34F8FBFF36F8FFEE700F09AF87F
:10A1A00000211046FFF72AFA00F06EFD002807D1C3
:10A1B00005494FF080500860BFF34F8FBFF36F8F9A
:10A1C00010BD00009809002004ED00E002498A6AF1
:10A1D00002604969416070479809002001490120E7
:10A1E000486270479809002010B50C4650B10949E3
:10A1F00009681831FFF7A1FE2046BDE81040012193
:10A20000FFF7FCB9502080F31188BFF34F8FBFF3E5
:10A210006F8FFEE79809002070B514460D4668B1AF
:10A220000A4909681831FFF7A0FE0CB14FF0FF355D
:10A2300021462846BDE87040FFF7E0B9502080F382
:10A240001188BFF34F8FBFF36F8FFEE7980900208F
:10A2500030B587B00025039505AA04A903A8049585
:10A26000FFF746FEDDE903010095CDE9011000236B
:10A2700014A11648059A00F0ECFB154C606318B168
:10A2800000F094FD012809D0401C19D1502080F322
:10A290001188BFF34F8FBFF36F8FFEE7502080F31D
:10A2A0001188BFF34F8FBFF36F8F4FF0FF302063E4
:10A2B0000120E061656107B0BDE8304000F068B89A
:10A2C00007B030BD49444C45000000009D9800088F
:10A2D000980900200248816B491C81637047000087
:10A2E00098090020164B10B5986B10B101205862E8
:10A2F00010BD002058629869124901E0B8B1401EB3
:10A3000000EB800251F82220002AF7D000EB8002F7
:10A3100001EB820101F108044A6852684A60A242D6
:10A3200001D152684A60D1681960986110BD50200F
:10A3300080F31188BFF34F8FBFF36F8FFEE70000EC
:10A3400098090020FC52002070B52020FFF72CFD5A
:10A35000040005D00025201D2560FFF7E0FD2577CE
:10A36000204670BD38B558B1202104460020009128
:10A370002060201DFFF7D3FD01202077204638BD47
:10A38000502080F31188BFF34F8FBFF36F8FFEE72C
:10A390001CB5264908780190FF20087008788DF8D0
:10A3A00000009DF800009DF8002000F0F0009042B1
:10A3B00007D0502080F31188BFF34F8FBFF36F8F0A
:10A3C000FEE79DF800001A4B00F0500018700720BF
:10A3D000986006E0401E98609DF8000040008DF8EF
:10A3E00000009DF8000000069868F3D4032807D009
:10A3F000502080F31188BFF34F8FBFF36F8FFEE7BC
:10A400004FF440709860019808700A48016841F460
:10A4100070010160016841F070410160FFF714FEB6
:10A4200000205860F5F7A0FE00201CBD00E400E00D
:10A43000040A002020ED00E010B50C4648B184422B
:10A440000FD9502080F31188BFF34F8FBFF36F8F68
:10A45000FEE7502080F31188BFF34F8FBFF36F8F5B
:10A46000FEE70222002100F03CF8002800D08463BF
:10A4700010BD38B50C4648B184420FD9502080F346
:10A480001188BFF34F8FBFF36F8FFEE7502080F32B
:10A490001188BFF34F8FBFF36F8FFEE70221134682
:10A4A00000220091114600F040F8002800D084639B
:10A4B00038BD10B502460021012000F012F8044614
:10A4C000FFF71CFA204610BD38B50B46002200905D
:10A4D0001146012000F029F80446FFF70FFA204644
:10A4E00038BDF8B517460E46050014D0DEB105FBA1
:10A4F00006F05030FFF758FC04000AD0002084F822
:10A50000460004F150023B46314628460094FFF7CE
:10A5100000FA2046F8BD502080F31188BFF34F8F1A
:10A52000BFF36F8FFEE70020E3E738B5049D18B155
:10A5300053B1CAB181B120E0502080F31188BFF33C
:10A540004F8FBFF36F8FFEE7502080F31188BFF36A
:10A550004F8FBFF36F8FFEE7502080F31188BFF35A
:10A560004F8FBFF36F8FFEE739B1502080F3118812
:10A57000BFF34F8FBFF36F8FFEE750241C460123BC
:10A5800084F846302B460094FFF7C3F9204638BDC7
:10A5900070B50D46040025D0FFF7F4FCD4E90F2078
:10A5A000216802FB001161600021A1632168A160A4
:10A5B0000A46D4E90F01401E00FB0121E16021465B
:10A5C0004FF0FF3001F8440F487004F110008DB1D6
:10A5D000FFF7A5FC04F12400FFF7A1FCFFF7F2FC54
:10A5E000012070BD502080F31188BFF34F8FBFF35F
:10A5F0006F8FFEE721690029F0D000F00DFB0028E5
:10A60000ECD004494FF080500860BFF34F8FBFF388
:10A610006F8FE3E704ED00E02DE9FF4F83B01F46A5
:10A620008B4604004FF0000603D0BBF1000F08D0AA
:10A6300011E0502080F31188BFF34F8FBFF36F8F6D
:10A64000FEE7206C38B1502080F31188BFF34F8FA4
:10A65000BFF36F8FFEE7022F0AD1E06B012807D00E
:10A66000502080F31188BFF34F8FBFF36F8FFEE749
:10A6700000F01CFADFF800914FF0000A4FF080580C
:10A6800048B9059838B1502080F31188BFF34F8F37
:10A69000BFF36F8FFEE7FFF775FCA06BE16B88429D
:10A6A00005D3022F03D00598C8B1DEB11EE03A46AB
:10A6B00059462046FFF77BF8616A19B104F124007E
:10A6C00000F0AAFA28B1C9F80080BFF34F8FBFF39A
:10A6D0006F8FFFF777FC012007B0BDE8F08FFFF721
:10A6E00071FC21E06846FFF771FD0126FFF76AFC67
:10A6F000FFF7F0FDFFF746FC94F94400401C01D140
:10A7000084F844A094F94500401C01D184F845A088
:10A71000FFF758FC05A9684600F02AF930B1204639
:10A72000FFF70CFB00F0B0FA0020D5E7FFF72AFC9A
:10A73000A06BE16B884201D1012500E00025FFF705
:10A7400041FC95B104F110000599FFF74DFD20463D
:10A75000FFF7F4FA00F098FA00289CD1C9F80080BD
:10A76000BFF34F8FBFF36F8F95E72046FFF7E6FAF1
:10A7700000F08AFA8FE7000004ED00E02DE9F047D1
:10A780001F4690468946040003D0B9F1000F08D057
:10A7900011E0502080F31188BFF34F8FBFF36F8F0C
:10A7A000FEE7206C38B1502080F31188BFF34F8F43
:10A7B000BFF36F8FFEE7022F0AD1E06B012807D0AD
:10A7C000502080F31188BFF34F8FBFF36F8FFEE7E8
:10A7D000FFF74CFC5020EFF3118680F31188BFF394
:10A7E0004F8FBFF36F8FA06BE16B884206D3022FB0
:10A7F00004D0002086F31188BDE8F08794F9455015
:10A800003A4649462046FEF7D2FF681C04D06D1C2C
:10A8100084F845500120EDE7606A0028FAD004F181
:10A82000240000F0F9F90028F4D0B8F1000FF1D0BD
:10A830000121C8F80010EDE72DE9F74783B08A46FB
:10A8400004004FF0000603D0BAF1000F08D011E069
:10A85000502080F31188BFF34F8FBFF36F8FFEE757
:10A86000206C38B1502080F31188BFF34F8FBFF3B5
:10A870006F8FFEE700F01AF9DFF8F09000274FF035
:10A88000805848B9059838B1502080F31188BFF33B
:10A890004F8FBFF36F8FFEE7FFF774FBA56BC5B15A
:10A8A00051462046FEF770FF6D1EA563206950B12A
:10A8B00004F1100000F0B0F928B1C9F80080BFF32E
:10A8C0004F8FBFF36F8FFFF77DFB012006B0BDE810
:10A8D000F087059808B11EB106E0FFF773FB27E08B
:10A8E0006846FFF773FC0126FFF76CFBFFF7F2FCED
:10A8F000FFF748FB94F94400401C01D184F84470F0
:10A9000094F94500401C01D184F84570FFF75AFBCB
:10A9100005A9684600F02CF8002820460AD0FFF769
:10A920000DFA00F0B1F92046FFF7B8F80028B3D0CF
:10A930000020CBE7FFF7B2F890B104F124000599AD
:10A94000FFF752FC2046FFF7F9F900F09DF90028C7
:10A95000A2D1C9F80080BFF34F8FBFF36F8F9BE781
:10A960002046FFF7EBF900F08FF995E704ED00E0E2
:10A970002DE9F0410C4605000FD0B4B1FFF702FB02
:10A980001C4E71696B683268C81A002792F85A2009
:10A990009AB1306880F85A701AE0502080F311881C
:10A9A000BFF34F8FBFF36F8FFEE7502080F3118806
:10A9B000BFF34F8FBFF36F8FFEE72268B2F1FF3F07
:10A9C00008D0D5F800C0B66AB44509D08B4207D884
:10A9D000012400E00024FFF7F5FA2046BDE8F081ED
:10A9E000824205D9101A20602846FFF7EFFBF1E7F5
:10A9F0002760EDE7980900202DE9FF5F8346DDE938
:10AA00000E87994616468A469000FFF7CDF9050055
:10AA10001CD05C20FFF7C8F9040014D00020256387
:10AA200084F85900CDE90240CDE900874B46324613
:10AA300051465846FEF77DFF2046FEF711FE0120E5
:10AA400004B0BDE8F09F2846FFF7D0FA4FF0FF3082
:10AA5000F6E7F0B585B00546DDE90B040A9EA8B11E
:10AA6000E4B15C2700972063022084F8590000209D
:10AA7000CDE9024004AF2846CDE90067FEF759FF53
:10AA80002046FEF7EDFD049805B0F0BD502080F3A0
:10AA90001188BFF34F8FBFF36F8FFEE7502080F315
:10AAA0001188BFF34F8FBFF36F8FFEE70548C16971
:10AAB00019B1806B18B10020704701207047022047
:10AAC0007047000098090020014840697047000065
:10AAD000980900202DE9F0412E4F0026B86B40B1B7
:10AAE000386A401C3862786A00B101263046BDE8F9
:10AAF000F0817D696D1C7D6113D17868006838B183
:10AB0000502080F31188BFF34F8FBFF36F8FFEE7A4
:10AB10007868B9687960B860B86A401CB862FFF7B5
:10AB20008BF8386BDFF87080854209D3786800684D
:10AB300080B17868C068C468606885420DD23863A7
:10AB40003868C06A00EB800158F821000128CAD992
:10AB50000126C8E74FF0FF30F1E7201DFFF7B4F9F9
:10AB6000A06A18B104F11800FFF7AEF9E06AB969FC
:10AB7000884200D9B86100EB800108EB8100211DFB
:10AB8000FFF7F3F9E06A3968C96A8842CED3012633
:10AB9000CCE7000098090020FC52002070B50400AA
:10ABA0004FF000002BD01A4D29688C4207D050205E
:10ABB00080F31188BFF34F8FBFF36F8FFEE7216DD6
:10ABC000F1B1491E2165E36CE26A9A4217D000296F
:10ABD00015D1201DFFF778F9E06CE062C0F1380074
:10ABE000A061E06AA969884200D9A861094900EB1F
:10ABF000800001EB8000211DFFF7B7F9012070BD37
:10AC0000502080F31188BFF34F8FBFF36F8FFEE7A3
:10AC100098090020FC52002070B5C068C46854B187
:10AC200004F118000646FFF74FF9144DA86B50B118
:10AC30003146134815E0502080F31188BFF34F8F41
:10AC4000BFF36F8FFEE7201DFFF73EF9E06AA969A9
:10AC5000884200D9A8610B4900EB800001EB80001D
:10AC6000211DFFF782F9E06A2968C96A884202D982
:10AC70000120686270BD002070BD000098090020AE
:10AC800084570020FC5200202DE9F0472B4D002472
:10AC90002746A86B38B1FFF775F9A86B401EA8636B
:10ACA000A86B40B145E0502080F31188BFF34F8F6F
:10ACB000BFF36F8FFEE7286921490126C8B3A1F5CC
:10ACC00091698846D8F80010E1B1D8F80C00C46842
:10ACD00004F11800FFF7F8F8201DFFF7F5F8E06A17
:10ACE000A969884200D9A86100EB800109EB8100C5
:10ACF000211DFFF73AF9E06A2968C96A8842E1D361
:10AD00006E62DFE70CB1FEF797FF2C6A3CB1FFF7EC
:10AD1000E1FE00B16E62641EF9D100202862686A0B
:10AD200038B10849012738070860BFF34F8FBFF3D8
:10AD30006F8FFFF747F93846BDE8F0879809002084
:10AD40008457002004ED00E02DE9FC4781461E46B3
:10AD50001746884630200A9DFFF726F804000AD0DF
:10AD6000CDE9005433463A4641464846FEF731FEA7
:10AD7000002084F82C002046BDE8FC877CB53025F7
:10AD8000DDE90664009544B1CDE90064FEF721FEDB
:10AD9000012084F82C0020467CBD502080F31188CF
:10ADA000BFF34F8FBFF36F8FFEE7000010B586B083
:10ADB000FEF7BEFC114CA068B8B1002003900490CF
:10ADC00005AA04A903A8FFF79DF8DDE903210220E5
:10ADD0008DE8070000230AA10B48059AFFF739FE0A
:10ADE000E06010B106B0012010BD502080F3118842
:10ADF000BFF34F8FBFF36F8FFEE70000D409002031
:10AE0000546D722053766300159D00082DE9FF41B3
:10AE10001F4603000A9E4FF0000015D0134DAC688A
:10AE2000002C0ED08DE80E00062917DAFFF73EFE43
:10AE300002284FF000030FD000226946A868FFF7F0
:10AE4000EBFB04B0BDE8F081502080F31188BFF324
:10AE50004F8FBFF36F8FFEE73246EEE700233A468F
:10AE600069462046FFF78AFCEBE70000D409002082
:10AE700000C1814001C0804101C0804100C18140CA
:10AE800001C0804100C1814000C1814001C08041BA
:10AE900001C0804100C1814000C1814001C08041AA
:10AEA00000C1814001C0804101C0804100C181409A
:10AEB00001C0804100C1814000C1814001C080418A
:10AEC00000C1814001C0804101C0804100C181407A
:10AED00000C1814001C0804101C0804100C181406A
:10AEE00001C0804100C1814000C1814001C080415A
:10AEF00001C0804100C1814000C1814001C080414A
:10AF000000C1814001C0804101C0804100C1814039
:10AF100000C1814001C0804101C0804100C1814029
:10AF200001C0804100C1814000C1814001C0804119
:10AF300000C1814001C0804101C0804100C1814009
:10AF400001C0804100C1814000C1814001C08041F9
:10AF500001C0804100C1814000C1814001C08041E9
:10AF600000C1814001C0804101C0804100C18140D9
:10AF700000C0C101C30302C2C60607C705C5C40499
:10AF8000CC0C0DCD0FCFCE0E0ACACB0BC90908C809
:10AF9000D81819D91BDBDA1A1EDEDF1FDD1D1CDCF9
:10AFA00014D4D515D71716D6D21213D311D1D01069
:10AFB000F03031F133F3F23236F6F737F53534F459
:10AFC0003CFCFD3DFF3F3EFEFA3A3BFB39F9F838C9
:10AFD00028E8E929EB2B2AEAEE2E2FEF2DEDEC2CB9
:10AFE000E42425E527E7E62622E2E323E12120E029
:10AFF000A06061A163A3A26266A6A767A56564A419
:10B000006CACAD6DAF6F6EAEAA6A6BAB69A9A86888
:10B0100078B8B979BB7B7ABABE7E7FBF7DBDBC7C78
:10B02000B47475B577B7B67672B2B373B17170B0E8
:10B0300050909151935352929656579755959454D8
:10B040009C5C5D9D5F9F9E5E5A9A9B5B9959589848
:10B05000884849894B8B8A4A4E8E8F4F8D4D4C8C38
:10B0600044848545874746868242438341818040A8
:10B070007CB8000800000000000000000000000094
:10B0800000000000000200001800000000000000A6
:10B0900000000000FCB500080000000000000000F7
:10B0A0000000000000000000000400000800000094
:10B0B000000000000000000078B60008000000005A
:10B0C000000000000000000000000000000400007C
:10B0D000080000000000000000000000E8B60008C2
:10B0E0000000000000000000000000000000000060
:10B0F0000004000008000000000000000000000044
:10B1000058B7000800000000000000000000000028
:10B110000000000000020000080000000000000025
:10B1200000000000A4B700080000000000000000BC
:10B130000000000000000000000200000800000005
:10B140000000000000000000E4B70008000000005C
:10B1500000000000000000000000000000020000ED
:10B1600008000000000000000000000024B80008F3
:10B1700000000000000000000000000000000000CF
:10B1800000020000080000000000000000000000B5
:10B1900064B800080000000000000000000000008B
:10B1A0000000000000020000080000000000000095
:10B1B0000000000068B5000800000000000000006A
:10B1C0000000000000000000000200000800000075
:10B1D0000000000000000000E4B5000800000000CE
:10B1E000000000000000000000000000000200005D
:10B1F00008000000000000000000000060B6000829
:10B20000000000000000000000000000000000003E
:10B21000000200000200000000000000000000002A
:10B2200080B50008000000000000000000000000E1
:10B230000000000000000000F0B500080000000061
:10B2400000000000000000000000000000000000FE
:10B250006CB60008000000000000000000000000C4
:10B260000000000000000000DCB600080000000044
:10B2700000000000000000000000000000000000CE
:10B280004CB70008000000000000000000000000B3
:10B29000000000000000000098B700080000000057
:10B2A000000000000000000000000000000000009E
:10B2B000ACB5000800000000000000000000000025
:10B2C00028B6000800000000000000000000000098
:10B2D000A4B600080000000000000000000000000C
:10B2E00014B700080000000000000000000000008B
:10B2F00074B700080000000000000000000000001B
:10B30000C0B70008000000000000000000000000BE
:10B3100000B800080000000000000000000000006D
:10B3200040B800080000000000000000000000001D
:10B3300070B80008000000000000000000000000DD
:10B3400074B50008000000000000000000000000CC
:10B35000D8B5000800000000000000000000000058
:10B3600054B60008000000000000000000000000CB
:10B37000D0B600080000000000000000000000003F
:10B3800040B70008000000000000000000000000BE
:10B390008CB7000800000000000000000000000062
:10B3A000D8B7000800000000000000000000000006
:10B3B00018B80008000000000000000000000000B5
:10B3C00058B8000800000000000000000000000065
:10B3D000C4B50008010000000000000000000000EB
:10B3E00040B600080100000000000000000000005E
:10B3F000BCB60008010000000000000000000000D2
:10B400002CB7000801000000000000000000000050
:10B410009CB50008000000000000000000000000D3
:10B4200018B6000800000000000000000000000046
:10B4300094B60008000000000000000000000000BA
:10B4400004B7000800000000000000000000000039
:10B4500064B70008000000000000000000000000C9
:10B46000B0B700080000000000000000000000006D
:10B47000F0B700080000000000000000000000001D
:10B4800030B80008000000000000000000000000CC
:10B490008CB5000800000000000000000000000063
:10B4A00008B60008000000000000000000000000D6
:10B4B00084B600080000000000000000000000004A
:10B4C000F4B60008000000000000000000000000CA
:10B4D000B8B50008000000000000000000000000F7
:10B4E00034B600080000000000000000000000006A
:10B4F000B0B60008000000000000000000000000DE
:10B5000020B700080000000000000000000000005C
:10B5100080B70008000000000000000000000000EC
:10B52000CCB7000800000000000000000000000090
:10B530000CB800080000000000000000000000003F
:10B540004CB80008000000000000000000000000EF
:10B5500000000000000000000102030406070809C3
:10B5600000000000010203046D795461736B3130F7
:10B57000000000006D7954696D6572313000000083
:10B580006D79517565756530310000006D79436FD7
:10B59000756E74696E6753656D3031006D794269FF
:10B5A0006E61727953656D30310000006D795469B8
:10B5B0006D657230310000006D794576656E7430CE
:10B5C000310000006D795265637572736976654D5F
:10B5D00075746578303100006D794D75746578301B
:10B5E000310000006D795461736B3131000000004F
:10B5F0006D79517565756530320000006D79546163
:10B60000736B3032000000006D79436F756E7469A2
:10B610006E6753656D3032006D7942696E61727983
:10B6200053656D30320000006D7954696D6572307C
:10B63000320000006D794576656E7430320000008E
:10B640006D795265637572736976654D7574657849
:10B65000303200006D794D7574657830320000002D
:10B660006D795461736B3132000000006D79517552
:10B6700065756530330000006D795461736B30334C
:10B68000000000006D79436F756E74696E675365D5
:10B690006D3033006D7942696E61727953656D303A
:10B6A000330000006D7954696D657230330000001D
:10B6B0006D794576656E7430330000006D795265A2
:10B6C000637572736976654D757465783033000003
:10B6D0006D794D7574657830330000006D79517562
:10B6E00065756530340000006D795461736B3034DA
:10B6F000000000006D79436F756E74696E67536565
:10B700006D3034006D7942696E61727953656D30C8
:10B71000340000006D7954696D65723034000000AA
:10B720006D794576656E7430340000006D79526530
:10B73000637572736976654D757465783034000091
:10B740006D794D7574657830340000006D795175F0
:10B7500065756530350000006D795461736B303567
:10B76000000000006D7942696E61727953656D3039
:10B77000350000006D7954696D6572303500000048
:10B780006D794576656E7430350000006D794D75C4
:10B7900074657830350000006D79517565756530D8
:10B7A000360000006D795461736B30360000000084
:10B7B0006D7942696E61727953656D3036000000B3
:10B7C0006D7954696D657230360000006D7945768B
:10B7D000656E7430360000006D794D757465783093
:10B7E000360000006D795461736B30370000000043
:10B7F0006D7942696E61727953656D303700000072
:10B800006D7954696D657230370000006D79457649
:10B81000656E7430370000006D794D757465783051
:10B82000370000006D795461736B30380000000000
:10B830006D7942696E61727953656D303800000030
:10B840006D7954696D657230380000006D79457608
:10B85000656E7430380000006D794D757465783010
:10B86000380000006D795461736B303900000000BE
:10B870006D7954696D6572303900000064656661E8
:10B88000756C745461736B00A8B800080000002048
:10B89000100A0000900800088CBE0008100A002062
:10B8A00080A50000908800082200010004FF0D0A16
:10B8B0000001910117110314100801000031030069
:10B8C00002025300E41010067103003D000C3281A7
:10B8D0001020079BCA51040A0F2013510435200879
:10B8E0001003AE61030004386148230139182007B2
:10B8F00055090300D0051700313EAA55AA5501028B
:10B90000030405060708090A0B0C0D0E0F1011128F
:10B91000131415161718191A1B1C1D1E1F2021227F
:10B92000232425262728292A2B2CC810098877AA02
:10B930009939019550BC21D20007ED009505AAAABE
:10B940000001340421032A0C540AAABBCCDDEEDD2D
:10B95000CCBB41D409361C2310040230069803499D
:10B9600007580200FF0077179817C017E117031850
:10B97000241845186A188F18B018D118F31814191C
:10B980003C195D197F19A019C119E6190B1A2C1A57
:10B990004D1A6F1A901AB81AD91AFB1A1C1B3D1BA4
:10B9A0005F1B801BA81BC91BEB1B0C1C2D1C4F1CF9
:10B9B000701C981CB91CDB1CFC1C1D1D3F1D601D50
:10B9C000811DA31DC41DEC1D0D1E2F1E501E711EBA
:10B9D000931EB41ED51EF71E181F391F5B1F7C1F38
:10B9E000971FB81FD91FFB1F1C203D205F20802000
:10B9F0009E20BC20DD20FF2020213E215C217D21D6
:10BA00009F21C021DB21FC211D22382259227B22CB
:10BA10009522B722D122F32214232F2350236B2304
:10BA20008C23AA23C823E32304241F2440245B245B
:10BA300075249724B324D124ED24082526254425F4
:10BA40005F257B259925B525D025EE250C262726B3
:10BA500043265C267A269826B126CD26E82603279B
:10BA60001F273827044F4256276F278827A627BF4E
:10BA700027D827F1270A281E283C2855286C288219
:10BA800028A028BE28D228E628FA280E292C2940EA
:10BA900029542968297C299029A429B829CC29E08E
:10BAA00029F429082A1C2A262A3A2A4E2A622A76AA
:10BAB0002A8A2A942AF014F269178B17B317D4171D
:10BAC000F5171718381859188118A318C418E5184D
:10BAD00007192F19501971199319B419D519FA1991
:10BAE0001F1A401A611A831AA41ACC1AED1A0F1BD6
:10BAF000301B511B731B941BBC1BDD1BFF1B201C2D
:10BB0000411C631C841CAC1CCD1CEF1C101D311D82
:10BB1000531D741D951DB71DD81DF91D1B1E3C1E00
:10BB2000641E851EA71EC81EE61E041F251F471F74
:10BB3000681F891FAB1FCC1FED1F0F2030204E2028
:10BB40006C208D20AF20D020F1200C212D214F2101
:10BB500070218B21AC21CD21E82109222B22452205
:10BB600067228822A322C422E22200231E233C2330
:10BB70005D2378239923B423D523F0230E242C248A
:10BB80004A2468248324A424BD24DB24F924152515
:10BB900030254E256C258725A325BC25DA25F825DB
:10BBA00011262D26482663267F921404B626CF92AE
:10BBB0009606927418A127BA27D327EC2705281CCC
:10BBC0002832284B28642878288828AD92941A2295
:10BBD0002936294A295E29722986299A29AE29C23D
:10BBE00029D629EA29FE29129406436C962D2003B2
:10BBF0002C07B917DB17FC1720033C0867188818B7
:10BC0000A918CE20033C06351957197820033C08A3
:10BC1000E319041A251A4720033C0AB11AD31AF46F
:10BC20001A151B3720031C0CA11BC31BE41B051C8E
:10BC3000271C482003741C911CB31CD41CF51C1732
:10BC40001D381D591D7B1D9C1DBD1DDF1D001E21A6
:10BC50001E43903412E91E0B1F2C1F4D1F6F1F90A7
:10BC60001FB11FD31FEF905406512073209490569C
:10BC7000139036919036EF90364C9056A6907621E0
:10BC80009016B9901408F723112431244D90168989
:10BC9000909C36C224E024FE241C253725532571B0
:10BCA000258D25A825C625DF25FD25192634264FF7
:10BCB000266B268426A226BB26D926F22610272903
:10BCC0002742275B2774278D220314062028372854
:10BCD00050909C067C289028AA24039E2224036569
:10BCE00090AD24033E582603063F80901C0669173A
:10BCF0008E17B6B0041C040918311E031E88AE044A
:10BD00001C06D8180019281C03258C1C04CF19F711
:10BD10001A031C0C471A721A9A1AC21AEA1A12A8A3
:10BD2000041406651B8D1BB5863C060C1C341C5C7C
:10BD300014031ED4A4041E2412031E7BA2041C049C
:10BD4000CB1DF310031C08461E6E1E961EBE0E036E
:10BD50001C0A0E1F361F5E1F861FAE9C04140401B2
:10BD600020297A14067920A120C9781414192141B8
:10BD70002169218E21B621DE2106222E2256227E25
:10BD8000721ECB92041C041B234390041A93FE1EC4
:10BD9000DC8E041C0A2C2454247C249D24C58A0493
:10BDA0001C0412253A88041C048725AF86041C1A3B
:10BDB000F8252026412669268E26B326DB26FC267A
:10BDC000242745276D278F27B77C041412002821CC
:10BDD0002846286B288C28B428D528F7281F4E1A07
:10BDE00061DC1EAB6C041AEDD61637400C89157950
:10BDF0002A9B2ABC2AE42A052B272B482B692B8B4C
:10BE00002BAC2BCD2BEF2B102C2B2C4C2C6D2C88F2
:10BE10002CA92CC42CEC2C0A2D322D502D6E2D8CDF
:10BE20002DAA2DC82DE62D042E222E402E5E2E7218
:10BE30002E9A2EAE2ECC2EEA2EFE2E1C2F3A2F58E6
:10BE40002F762F8A2F9E2FBC2FDA2FEE2F02302035
:10BE5000303E30523066307A308E30A230C030D42E
:10BE600030E830FC30103124313831423156316AFB
:10BE7000317E3192319C31B9043F24F43B080E7578
:0CBE80001028074FAAAA1C0800000000B0
:0400000508000131BD
:00000001FF
